:1000000023C3000059C3000057C3000055C30000BC
:1000100053C3000051C300004FC300004DC3000094
:100020004BC3000049C300000C949C310C948432F3
:100030000C94513141C300003FC300003DC3000098
:100040003BC3000039C3000037C3000035C30000C4
:1000500033C300000C9478312FC300002DC300007F
:100060002BC3000029C3000027C3000025C30000E4
:1000700023C3000021C300001FC300001DC30000F4
:100080001BC3000019C3000017C3000015C3000004
:1000900013C3000011C300000FC300000DC3000014
:1000A0000BC3000009C3000007C30000050109805D
:1000B000A101850319012AB700150126B700950192
:1000C00075108100C0050C0901A101850419012AE0
:1000D000A002150126A002950175108100C005013E
:1000E0000906A1018506050719E029E71500250184
:1000F0009508750181020507190029EF15002501F2
:1001000095F075018102050819012905950575010C
:100110009102950175039101C00660FF0961A1017B
:100120000962150026FF00952075088102096315F4
:100130000026FF00952075089102C005010906A15F
:1001400001050719E029E7150025019508750181CA
:10015000029501750881010507190029FF15002680
:10016000FF0095067508810005081901290515008D
:100170002501950575019102950175039101C00056
:10018000000000000000000000000000000000006F
:10019000000000000000000000000000000000005F
:1001A0000000007E0F00D4FFFFFFC70000007800B2
:1001B000000000000000002A2B28000000000000C2
:1001C0000000000000000000000029000000002CDA
:1001D0001E3420212224342627252E362D37382779
:1001E0001E1F202122232425263333362E37381F85
:1001F0000405060708090A0B0C0D0E0F1011121347
:100200001415161718191A1B1C1D2F3130232D35E4
:100210000405060708090A0B0C0D0E0F1011121326
:100220001415161718191A1B1C1D2F3130354C09BF
:10023000025B00030100A0FA0904000001030101B0
:100240000009211101000122440007058103080073
:10025000010904010002030000000921110100014D
:100260002222000705820320000107050303200066
:10027000010904020001030000000921110100012D
:10028000226D000705840320000112010002000016
:1002900000081502E3120001010203011C037600AD
:1002A000690061006C003A006600360034006300AB
:1002B0003200620033006300000020036300780016
:1002C00074005F00730074007500640069006F00C3
:1002D00020003100320045003300000016036300A7
:1002E000780074005F00730074007500640069009A
:1002F0006F0000000403090429001B010601190115
:1003000046001D01B200AB002152E3004C00650025
:100310000000AE00D30042784378477849004C0093
:10032000447848784B004A000100007C4E004D00A4
:100330000000A80001000100D900DA004B004E00C7
:10034000A900AA00457846784B784C7849784A78D5
:100350000001010101010101010102020202020288
:10036000020202030303030303030304040404045B
:100370000404050505050506060606060707070722
:100380000708080808090909090A0A0A0B0B0B0CD7
:100390000C0C0D0D0D0E0E0E0F0F0F101011111174
:1003A00012121313141415151616171718181919F5
:1003B0001A1A1B1B1C1D1D1E1E1F2020212222235A
:1003C0002424252626272829292A2B2C2D2D2E2F9B
:1003D00030313232333435363738393A3B3C3D3EB2
:1003E0003F404142434445464748494A4C4D4E4FA1
:1003F00050515354555658595A5B5D5E5F61626463
:10040000656668696B6C6D6F7072737577787A7BEF
:100410007D7E8082838587888A8C8E8F9193959646
:10042000989A9C9EA0A2A3A5A7A9ABADAFB1B3B566
:10043000B7BABCBEC0C2C4C6C9CBCDCFD1D4D6D842
:10044000DBDDDFE2E4E7E9EBEEF0F3F5F8FAFDFFE0
:1004500001000100B204E9273D280000020002006B
:10046000AE04E9273D28000003000100B304E9279A
:100470003D280000040002009804E9273D28AE074B
:1004800005000100B404E9273D2800000600020031
:100490009A04E9273D28000007000200B004E9277C
:1004A0003D28000012000200B604E9273D280000A4
:1004B00013000200B804E9273D28000014000100E1
:1004C000BA04E9273D280000150000000000B70726
:1004D000190E000016000100B50400285528000080
:1004E00017000101B504002855280000180001027A
:1004F000B50400285528000019000200BC04E927B3
:100500003D2800001A000103B5040028552800000A
:100510001B000200BE04E9273D280000FD377A5881
:100520005A000004E6D6B44602002101160000007D
:10053000742FE5A3E001D000DC5D003D8889C6543E
:1005400036C3174FE4EFB3D58A10B65DAF2D2AF24C
:100550008121B9609E20D04B074DE39D2DE5C42637
:10056000C8C0663536E3DE00E4FBBAD2A4E75D9C82
:1005700035F764EC7F6D436E3A8EFB94FA0D1D5196
:100580002FBC443F6B11200F4FF2DA7AC408D68398
:10059000B4D551FE9D5DD9EBE32B7A63BFF3D71F32
:1005A000969B7B8F0BE80120B344535EBD0B56AD89
:1005B00085FFFA0FE3E0641BFF1C38D6CA8A1B7D57
:1005C000610E71C51BD4B0D52A443505AC3D88C336
:1005D00028820836B778A8CB55A7EFD82FE6AD47C5
:1005E000851F3A38F0DDCDE6F7AC5BFF607F473220
:1005F000C70F89BEF141CC1725046E87B3FE735136
:1006000088BDF46D705B5270CD9938A488015D5D32
:100610005AFBFAAD9F007E0020914E2CA402B3F548
:100620000001F801D1030000BC065A9BB1C467FB6E
:10063000020000000004595A4C2A52524C2A5252CD
:100640004C2A52520052525211241FBECFEFDAE010
:10065000DEBFCDBF04B603FE18C080913C0590916B
:100660003D05A0913E05B0913F058730904BA740D6
:10067000B04B59F410923C0510923D0510923E0586
:1006800010923F05E0E0F8E3099512E0A0E0B1E048
:10069000ECE0F8E602C005900D92A430B107D9F75E
:1006A00025E0A4E0B2E001C01D92AC33B207E1F74F
:1006B0000E946A290C94C133A3CC9C01FB019A953A
:1006C00081159F4120F5832F8170B32FB270AA2727
:1006D000732F74706627532F5870442734FF0DC052
:1006E0008295807FAB2B09F08062672B09F08064D4
:1006F000452B09F0806809950895AB2B09F08260BD
:10070000672B09F08460452BB1F38860F4CF80E05B
:10071000F2CF982F92959F7024E0911102C020E0B3
:10072000982F892F86958695811511F02E5F982F29
:10073000892F8695820F0895282F92959F70963065
:1007400099F060F4925F9F70923030F4203FB1F0E6
:1007500038F481E0283E38F080E008959A5FF3CFC6
:1007600081E0243FC9F7089591E0813F09F090E0CE
:1007700081E0283E08F080E0892B089581E008950B
:1007800080933705089580933805089521E030E07F
:1007900001C0220F8A95EAF780913805822BF3CFAA
:1007A00021E030E0A90102C0440F551F8A95E2F70D
:1007B000CA018095909138058923E5CF9B01677028
:1007C00091E001C0990F6A95EAF763E036952795A5
:1007D0006A95E1F7B901660F771F260F371FFA01F7
:1007E000E20FF31F40E050E0682F70E08191DF01DD
:1007F0009B01042E02C0369527950A94E2F72170DA
:1008000021952827292328272E934F5F5F4F4330B8
:10081000510561F708959C01A82FA77083E03695D4
:1008200027958A95E1F7C901880F991F820F931FB9
:10083000FB01E80FF91F40E050E080E0219130E03B
:100840000A2E02C0369527950A94E2F721703327C5
:10085000042E01C0220F0A94EAF7822B4F5F5F4FEC
:100860004330510559F70895282F862F903F69F09E
:10087000943060F4243048F434E0939FB0011124A4
:10088000620F711D4DEA53E099CF08959C5F92303D
:10089000E0F7622F70E04AEA53E0F6CF282F903F4E
:1008A000A1F0943058F4843080F434E0939FC00178
:1008B00011246DEA73E0820F911DADCF9C5F9230E1
:1008C00020F46AEA73E090E0F8CF80E00895909118
:1008D000380521E030E0F90101C0EE0F8A95EAF712
:1008E000D90102C0AA0FBB1F6A95E2F7EA2B01C02B
:1008F000220F4A95EAF7892F8E23E81303C0892F28
:10090000822B41CF2095822F8923FBCF80916103D9
:1009100090E020E0022E001C0008281709060CF0C9
:1009200008952F5FF7CFCF93DF93EC01DB018C812C
:10093000813059F514968C911497813031F5E98105
:1009400084E0E89FF00111248881E80FF11DE85C44
:10095000F94F94919A32C9F01196EC91119784E075
:10096000E89FF00111248C91E80FF11DE85CF94F2C
:10097000E49181E09E1301C080E091E0EA3209F049
:1009800090E0892BDF91CF91089581E0FBCF9C010E
:1009900080915C048D79811119C0211540E53407DF
:1009A00080F4211580E23807C0F42333310511F1BA
:1009B000D0F481E02E31310590F42430310530F04F
:1009C0000895C90196558115914010F080E0089571
:1009D000C901805F96450797C8F33327E6CF2C32CD
:1009E0003105A1F708952653310981E023303105FF
:1009F00038F3ECCF81E008958091C3039091C20356
:100A0000981301C008958F5F8770FACF90915C04AE
:100A1000982B90935C040895982F909580915C0496
:100A2000892380935C040895982F909580915F04AA
:100A3000892380935F040895811520E59207C0F50E
:100A4000811540E4940708F0A0C0833C9105A0F410
:100A5000883A910508F08CC0853A910550F48430AD
:100A6000910510F521E0019709F020E0822F90E038
:100A70000895849790640895811560E29607A8F41C
:100A8000811571E0970780F4803E910538F48D3C24
:100A9000910508F078C080E090E008959C01205E08
:100AA000310928303105B8F708959F719062089593
:100AB000803622E5920740F5803442E5940708F03D
:100AC0007CC0803262E59607C0F4811572E5970715
:100AD00008F05EC09C0163E0220F331F6A95E1F7C6
:100AE00022273F70682F6F71462F50E084FD80C031
:100AF000242B352BC901906908958F7190E0982FB0
:100B00008827816F906A0895803C22E5920710F54E
:100B1000803A42E5940708F066C09C0120563245B1
:100B20002032310508F0B7CF282F2695269527705B
:100B300070E2279F90011124837041E050E0BA01D8
:100B400002C0660F771F8A95E2F7CB01822B932BA9
:100B50009A6808959C01205C32452032310508F0E6
:100B60009ACF982F882788279F71806F906A089561
:100B7000885AE82FF0E0EE0FFF1FE956FE4F808104
:100B8000918194640895906508959F70906A089586
:100B9000282F2695269560E2269F900111248370C8
:100BA00041E050E0BA0102C0660F771F8A95E2F774
:100BB000CB01822B932B9D680895282F269526958F
:100BC000277070E2279F90011124837041E050E06C
:100BD000BA0102C0660F771F8A95E2F7CB01822B1C
:100BE000932B9C6808958F7190E0982F8827089523
:100BF00070E1679FA001112455277ACF80E0089506
:100C0000F894E82FE295EF70F0E041A18F7021E0B9
:100C100030E0B90102C0660F771F8A95E2F7CB0179
:100C2000962F9095942391A392A1892B82A37894D7
:100C30000895CF92DF92EF92FF921F93CF93DF93AD
:100C4000172FE82FF0E0E05BFC4F71110CC0E4912E
:100C50008E2F7E2F6E2FDF91CF911F91FF90EF90FF
:100C6000DF90CF900895E62EF12CC72ED12CF49171
:100C7000EF2F86E0689F90011124CFEFD0E0C901EB
:100C8000BE010E940633AB01EE0CFF1C65E5649FBC
:100C9000C001659F900D1124E81AF90A6E2D660FA8
:100CA0006E0D7E01EC18FD08FE9DD001FF9DB00D7C
:100CB00011248B2F169F70011124EF2CFF246E013D
:100CC000CE18DF087601FE9D6001FF9DD00C112437
:100CD0007E01E61AF108B701169F7001179FF00C0C
:100CE0001124EF2CFF24CE19DF09FC9F7001FD9F1A
:100CF000F00C11247F2D43305105C1F02C3F3340BF
:100D000058F441305105B1F04230510509F0A2CFFD
:100D1000EB2F8F2D7F2F9ECF4430510571F0463041
:100D2000510509F497CF7B2F8D2D94CF7D2DEB2F7F
:100D30008F2F90CF7F2FED2D8DCFEF2D7B2FF8CFE5
:100D4000482F2695E22F26FDE0959E2F9F7026FDC9
:100D50009F5FE695E695E695E670F0E0E059FE4F78
:100D60003181399F302D912D112432953F7092950C
:100D7000907F392B9081930F27FD919597FD919549
:100D8000990F292F249F020E20E0211D1124822F6C
:100D900008959091F502982B9093F5020895A5C1BE
:100DA0000895E2E1F3E0808191E089278083109249
:100DB000050181E0EECF809112038370811102C0A2
:100DC00010920501809112038C7F81608093120341
:100DD0000895809112038370811110920501809112
:100DE00012038C7F809312030895982F862F2091F1
:100DF00012032370211581F0911579F0933078F466
:100E00009F73990F990F209112032370922B909347
:100E1000120310920501BDCF089591E0F2CF92E048
:100E2000F0CF80911203869586958F5F833008F00E
:100E300081E061E0DACF80911203869586958A95EC
:100E400009F482E061E0D1CF982F822F2091120324
:100E50002370211539F0909313036093140340938A
:100E6000150397CF0895E2E1F3E0818190E021E05E
:100E7000438162810896E8CFE2E1F3E0818121E0DD
:100E8000438162818850990BDFCFE2E1F3E0628118
:100E900020E1620F08F46FEF818121E0438190E04F
:100EA000D3CFE2E1F3E0628120E1621B08F460E06D
:100EB000818121E0438190E0C7CFE2E1F3E043810B
:100EC00020E1420F08F44FEF818121E0628190E040
:100ED000BBCFE2E1F3E0438120E1421B08F440E0B4
:100EE000818121E0628190E0AFCFE2E1F3E02481F3
:100EF00030E1230F08F42FEF248381E04ACFE2E1B1
:100F0000F3E0248130E1231B08F420E0248381E016
:100F100040CF81152CE7920741F420911E033091B8
:100F20001F03232B11F480E090E00895E2EDF3E03D
:100F300080E090E065E775E248E955E22AE036E2B4
:100F40007683658350874783328721879687858795
:100F500001963F968830910599F7089580919804FD
:100F60009091990490931301809312010895EF9248
:100F7000FF920F931F93CF93DF93FB018FEF9FEFB0
:100F80004430510508F45FC04091B30341FB88270A
:100F900080F990E0880F991F42FB002700F910E0CC
:100FA000000F111F000F111F802B912B40FBEE240F
:100FB000E0F8F12C8E299F2943FB222720F9C22F2C
:100FC00050E0D52F53E0CC0FDD1F5A95E1F78C2B65
:100FD0009D2B44FB222720F950E1259F90011124ED
:100FE000822B932B45FB222720F950E2259F90016D
:100FF0001124822B932B46FB222720F950E4259FB6
:1010000090011124822B932B47FB222720F940E8E3
:10101000249F90011124822B932B2091B403322F13
:101020003170932B26952170B22FBB0FA0E08A2B35
:101030009B2B092E000CAA0BBB0B80839183A283F0
:10104000B38380E090E0CDB7DEB7E6E00C94F732F2
:1010500090E06115E9F0875C9E4FFC0180818F3F35
:10106000B1F0E82FE295EF70F0E041A18F7021E040
:1010700030E0B90102C0660F771F8A95E2F7CB0115
:10108000962F9095942391A392A1892B82A30895E2
:101090008A5C9E4FE2CF90E06115A9F0875C9E4F7D
:1010A000FC0120812F3F91F0E22FE295EF70E05E8E
:1010B000F0E0808190E02F7002C0959587952A9589
:1010C000E2F7817008958A5C9E4FEACF80E0089530
:1010D000879A0895FC01EE0FFF1FE80FF91FE359EF
:1010E000FD4F6183408322830895FF920F931F93E6
:1010F000CF93DF93182F062FF42EC0E0D0E02F2DD2
:10110000402F612FCE01E6DF2196CC30D105B9F713
:10111000CDB7DEB7E5E00C94F832AC0123E096954C
:1011200087952A95E1F78E719927FC01E35BFD4FC6
:101130000190F081E02D4F70552721E030E002C092
:10114000220F331F4A95E2F7611541F0E22BF32B92
:10115000835B9D4FDC01ED93FC93089520953095C2
:10116000E223F323F5CF1092C9041092C804E0E6FD
:10117000F4E08581811102C014821682379684E0E2
:10118000E839F807B1F70895AC013091CB046091CC
:10119000CA04232F621301C00895822F90E0FC013E
:1011A000EE0FFF1FE054FB4F0190F081E02DE4179C
:1011B000F50791F467E0649FF001659FF00D11243D
:1011C000E05AFB4F41E044832313E6CF019683703E
:1011D00099278093CB0408950196282F2370DACFA6
:1011E0000F931F93CF9301E010E0082E01C0000F72
:1011F0000A94EAF7C0915B049C2F9023911108C0D8
:10120000C5DAC027C0935B04CF911F910F91089559
:10121000C7DAF7CFFA01309709F009950895E09100
:101220004703F0914803309739F00190F081E02DA9
:10123000309711F00995089580E00895A3E0B0E09B
:10124000E4E2F9E00C94DF329C0180914A02909133
:101250004B0282179307B1F030934B0220934A025E
:10126000E0914703F0914803309761F00084F185E5
:10127000E02D309739F083E089833B832A83CE01C8
:10128000019609952396E2E00C94FB32A3E0B0E0CE
:10129000ECE4F9E00C94DF329C01809148029091DB
:1012A000490282179307B1F0309349022093480214
:1012B000E0914703F0914803309761F00084F18595
:1012C000E02D309739F084E089833B832A83CE0177
:1012D000019609952396E2E00C94FB329091160159
:1012E000913021F49091B30397FD0CC0E8E0F2E057
:1012F0009191891302C0DF011E9252E0EE30F50792
:10130000B9F70895E82FE695E695E695803FC8F78A
:10131000F0E0E25FFD4F877021E030E0A90102C0FC
:10132000440F551F8A95E2F7CA018095928189235F
:10133000828308958091150108952FB7F8948091C4
:10134000440290914502A0914602B09147022FBFFE
:1013500008952FB7F89460914402709145028091EE
:101360004602909147022FBF08950895FC019B010A
:1013700080913A0290913B028617970740F0672BC5
:1013800029F48091E8008E778093E800C90140E05D
:10139000009741F4411106C08091E80082FF2FC000
:1013A00080E00895209120032115A9F12530A9F1AD
:1013B0002091E80023FD2DC02091E80022FDECCF14
:1013C0002091E80020FFE4CF3091F3002091F2005B
:1013D000009719F02830310558F041E028303105E8
:1013E00009F040E02091E8002E772093E800D0CF6C
:1013F00041914093F10001972F5F3F4FE9CF8091DA
:101400002003811541F0853041F08091E80083FF91
:10141000C3CF81E0089582E0089583E0089580912C
:10142000340287FF13C08091E80082FF06C08091DC
:10143000E8008B778093E800089580912003811164
:10144000F2CF0895809120038115D9F38091E800AF
:1014500080FFF8CF8091E8008E77ECCF2091E400F8
:101460003091E50095E6A9012091EC00822F817072
:1014700020FF06C08091E80080FF06C080E008954C
:101480002091E80022FD1AC080912003811589F087
:10149000853089F08091EB0085FD0FC02091E4003C
:1014A0003091E50042175307F9F29A95E1F684E08E
:1014B000089582E0089583E0089581E00895E8EDBD
:1014C000F0E080818E7F80831092E2001092DA003B
:1014D0001092E100A0EEB0E08C9181608C9380814D
:1014E0008F77808319BCA7EDB0E08C918E7F8C93B1
:1014F00080818F7E8083109233020895E0914703AC
:10150000F0914803309739F00284F385E02D30974D
:1015100011F060E209950895982F9093E9008917DA
:1015200071F07091EC002091ED005091F00021FDE0
:1015300009C09F5F973089F78093E9000895762F5F
:10154000242F50E03091EB003E7F3093EB00309140
:10155000ED003D7F3093ED003091EB003160309332
:10156000EB007093EC002093ED005093F00020917D
:10157000EE0027FDDECF0895A0E0B0E0E2ECFAE057
:101580000C94D932C8EDD0E088818F7E8883E7ED56
:10159000F0E080818160808384E082BF81E080937D
:1015A000330288818E7F888302EE10E0F80110827A
:1015B0001092DA0081EEC82ED12CF60110828881BB
:1015C0008F77888388818068888388818F7D8883EE
:1015D00019BC10922003109232021092F70210925E
:1015E000310290EEE92EF12CF70180818B7F808310
:1015F00088818160888342E060E080E08DDFF601D1
:1016000080818E7F8083F8018081816080838081EA
:1016100088608083F70180818E7F808388818061EC
:101620008883CDB7DEB7E8E00C94F532E091C303D0
:101630009091C20329E0E91302C080E00895AE2F23
:10164000B0E02E9FF0011124EE59FC4F318136138A
:1016500006C03081381303C03581341304C0FD0146
:101660003196E770E8CF81E008959C01211531059E
:1016700009F408958FE99FE00197F1F700C0000099
:1016800021503109F3CF31B33F7721B320684FB7F1
:10169000F8948DE692E0FC010196508168E021BB50
:1016A000000000C057FF31BB550F000000C000C054
:1016B00000C031BB00C06A9591F752E081399507AF
:1016C00051F74FBF8FE594E00197F1F700C000009C
:1016D000089581E08093E00080E28093D80010922A
:1016E000C9008FE19EE40197F1F700C0000087E098
:1016F00090EBDC0180933C0590933D05A0933E0563
:10170000B0933F0588E19CE00FB6F894A8958093CC
:1017100060000FBE90936000FFCF0F931F93CF9395
:10172000DF938B01EA0190912003943051F580936F
:10173000E9008FEF9091E80095FD06C095ED9A9530
:10174000F1F700008A95B1F78091E80085FF19C094
:1017500085DE811111C08091E80085FD06C0809171
:10176000E8008E778093E800F3CFF80181918F0134
:101770008093F100219779F78091E8008E7780932C
:10178000E800DF91CF911F910F910895792F60327A
:1017900029F440E250E0682F82E0BFCF0895CF9354
:1017A000DF93D82FC92F48E050E0682F792F81E0D0
:1017B000B4DF88E0ED2FFC2FACE3B2E001900D9296
:1017C0008A95E1F7DF91CF910895BC0140E250E0A6
:1017D00084E0A3CFBC0143E050E084E09ECF1F93A0
:1017E000CF93DF93C62F122F632F9C2F942B982B10
:1017F0009430B8F428E0C29FE0011124C40FD11D39
:10180000C40FD11D20E2829FC0011124C80FD91F2F
:10181000CE0189960E948C33612FCE018A960E9458
:101820008C33DF91CF911F9108950F931F93CF9326
:10183000DF93C62F142F022F632F843010F5C3308F
:1018400000F524E0C29FE00111243CE0839FC00D1D
:10185000D11D1124C755DF4F81E084279E01280F39
:10186000311D280F311DC9010E948C3381E090E0A9
:10187000111102C083E090E0602F8C0F9D1F0E9429
:101880008C33DF91CF911F910F91089580915F0468
:1018900090915C04892B90911601913059F59091AB
:1018A000B30397FF27C080930F0240E250E067E246
:1018B00073E08EE092E00E944333892BD1F080E206
:1018C000EEE0F2E0A7E2B3E001900D928A95E1F735
:1018D000E0914703F0914803309759F00480F58177
:1018E000E02D309731F086E080930E028EE092E09A
:1018F000099508958093060248E050E069E473E09A
:1019000086E092E00E944333892B99F388E0E6E079
:10191000F2E0A9E4B3E001900D928A95E1F7E0913D
:101920004703F0914803309721F30280F381E02DC3
:101930003097F9F286E092E0DBCF811511F066D89E
:10194000A5CF0895811531F090915F04892B809384
:101950005F049CCF0895811511F05ED897CF08954C
:10196000811511F061D892CF08958091CE03811531
:1019700021F082E2F5DF1092CE030895CF93C82FB5
:10198000811509F468C08CEF8C0F813A08F065C0AE
:1019900080911601813041F1E8E0F2E08EE092E0C2
:1019A0002191C217D9F18E179F07D1F780911601A7
:1019B0008130C1F1A8E0B2E0EFEF80E09D91C9175E
:1019C00009F448C0EF3F19F4911101C0E82F8F5F6F
:1019D0008630A1F7EF3F09F43DC00E2E000CFF0B3F
:1019E000EA5FFD4FC28336C08091B30387FFD4CF37
:1019F000EC2FE695E695E695F0E0E25FFD4F8281FB
:101A000090E04C2F477021E030E002C0220F331FDE
:101A10004A95E2F782239323892B21F08C2F5EDCF9
:101A200035DFC4CF8091B30387FFC4CFAC2FA69519
:101A3000A695A695B0E0A25FBD4FC77081E090E08B
:101A400001C0880FCA95EAF71296CC911297C82B5D
:101A50001296CC931BDFCF91089580E28C0F8830D3
:101A600048F4C77081E001C0880FCA95EAF70E9468
:101A70000605F0CF8BE58C0F833030F42C2F2452E9
:101A8000330BC901DBDBE7CFC85ACB3120F7EC2F92
:101A9000F0E0EE0FFF1FE353FE4F80819181F6DBF4
:101AA000DACFCF93DF93EC01805E9109089720F0A5
:101AB00062EA7CE0209711F46DE97CE0CE010E949F
:101AC0005D038C2F5BDFDF91CF910895611529F0C5
:101AD00020915F04226020935F049C013052211505
:101AE000304308F49927DDCF811509F19CEF980F59
:101AF000913A10F4F3DBCACE90E2980F983050F48C
:101B0000877091E001C0990F8A95EAF7892F0E94AA
:101B10000C05F1CF9BE5980F933018F480E090E02E
:101B20008DCB885A8B3118F480E090E0AFCB0895CC
:101B3000CF93DF93EC01D8DFCE01805E9109089747
:101B400020F060EB7CE0209711F46BEA7CE0CE01A2
:101B50000E945D03DF91CF9108951F93CF93DF9390
:101B6000182FEB010BDF209731F4812FBDDFDF91C0
:101B7000CF911F9108958FE99FE00197F1F700C081
:101B800000002197F0CF6091B8047091B9048933B7
:101B900021F06091B6047091B704DFCF10925C041D
:101BA000809116018130A1F48091B30387FF10C0AA
:101BB000E0E1F2E08EE1DF011D928A95E9F780E035
:101BC00090E03CDB80E090E061DB10925F045ECE51
:101BD000E8E0F2E086E0EFCFE1DF2FEF84E39CE086
:101BE000215080409040E1F700C0000088E19CE077
:101BF0000FB6F894A895809360000FBE9093600094
:101C0000FFCFCF93DF93D82FC92F209161032830C6
:101C100010F0C4DF20E0E22FF0E0EE0FFF1FEF5ADC
:101C2000FC4FD083C1832F5F20936103DF91CF915D
:101C30000895CF93DF93FB018FEF9FEF4430510561
:101C4000B0F0D081C181AADFD093B303C37080917B
:101C5000B4038C7FC82BC093B4036091B30370911D
:101C6000B40384E090E00E94A63380E090E0DF912E
:101C7000CF910895AAE2B0E0E0E4FEE00C94DE32F9
:101C800084E392E0FC0101962091F100208322E0A0
:101C90008C339207B9F780913502893009F457C027
:101CA000C8F4823009F4B2C0833009F482C08130B4
:101CB00081F18091E80083FFE6C080913402909129
:101CC00035029A3008F0DFC0E92FF0E0ED53FC4C0C
:101CD0000C942D338A3009F489C08B3051F78091F0
:101CE0003402813231F78091380290913902892B88
:101CF00001F78091E800877F8093E80090DB81E026
:101D000090913602911101C080E08093160146DF68
:101D1000D0CF80913402813A61F68091E800877FCC
:101D20008093E8008091380290913902892B59F014
:101D300060E080E090E070E019DB8091E8008B7754
:101D40008093E800B6CF68E08CE392E0F4CF809116
:101D50003402813209F0ADCF80913802909139027E
:101D60008D7F892B09F0A5CF8091E800877F809334
:101D7000E8008091E80082FF17C09091F300809105
:101D8000F200029731F48091F100813011F0863039
:101D900021F48091F100809315018091E8008B7708
:101DA0008093E8003CDB85CF809120038111E1CF57
:101DB00080CF80913402813A09F07BCF8091380244
:101DC00090913902892B09F074CF8091E800877FC8
:101DD0008093E8008091E80080FFFCCF809116019D
:101DE0008093F1008091E8008E77DACF8091340201
:101DF000813209F05ECF8091E800877F8093E80010
:101E00000EDB809137028093140153CF809134020E
:101E1000813A09F04ECF8091E800877F8093E800F7
:101E20008091E80080FFFCCF80911401D9CF8038E9
:101E300089F0823841F5809138028F70873018F52B
:101E40008093E9008091EB0085FB882780F9109250
:101E5000E90006C08091F702880F90913102892B2A
:101E60009091E800977F9093E8008093F1001092A2
:101E7000F1008091E8008E7723C0811116C0809117
:101E80003602813009F18091E80083FF0AC0809119
:101E9000E800877F8093E8008091EB008062809368
:101EA000EB00AA96E3E00C94FA32823061F780915D
:101EB0003602811581F01092E9008091E800877F59
:101EC0008093E800ACDADFCF81E0933009F080E066
:101ED0008093F702F0CF809138028F702FEF280F98
:101EE000263088F68093E9002091EB0020FFE3CFB5
:101EF000933031F48091EB0080628093EB00DBCF74
:101F00009091EB0090619093EB0021E030E0A9010B
:101F100002C0440F551F8A95E2F74093EA001092E1
:101F2000EA008091EB008860E8CF8111ACCF10917E
:101F300036021F778091E3008078812B8093E30045
:101F40008091E800877F8093E80069DA8091E8005B
:101F500080FFFCCF8091E30080688093E30083E002
:101F6000111101C082E0809320038DCF8058823010
:101F700008F089CF80913602909137028C3D53E072
:101F8000950791F583E08A838AE289834FB7F894B5
:101F9000DE01139620E03EE051E2E32FF0E05093A3
:101FA0005700849120FF03C082958F703F5F8F7030
:101FB0008A30C0F0895C90E08D939D932F5F24312F
:101FC00061F74FBF8091E800877F8093E8006AE265
:101FD00070E0CE010196CAD98091E8008B7780939A
:101FE000E80051CF805DE7CF292F3327233031051B
:101FF00009F44EC078F52130310509F488C08BE52D
:1020000090E0EFE2F2E02230310509F03CCF209180
:10201000E800277F2093E80020913A0230913B02AC
:102020008217930708F49C0140E02115310509F05F
:1020300073C0411171C08091E80082FDCDCF8091C5
:102040002003811549F2853039F28091E80083FF41
:10205000F2CFC2CF809138029091390221323105FE
:1020600009F446C02232310509F00DCF83309105C5
:1020700008F009CFFC01EE0FFF1FE65DFE4F019057
:10208000F081E02D895D9E4FDC018C9190E010C0C5
:102090009C013327823021F12330310568F4232B52
:1020A000B9F4E4EFF2E0E4918E2F90E0E4EFF2E097
:1020B000009709F4E8CEABCF2330310509F0E3CE29
:1020C000ECE9F2E0E4918E2F90E0ECE9F2E0F0CF61
:1020D000ECEDF2E0E4918E2F90E0ECEDF2E0E8CF51
:1020E000EAEBF2E0E4918E2F90E0EAEBF2E0E0CF51
:1020F0008330910508F0C7CEFC01EE0FFF1FE05DB5
:10210000FE4F0190F081E02D89E090E080CF82E1E8
:1021100090E0EAE8F2E07BCF80912003811509F49A
:102120005BCF853009F458CF8091E80083FD54CF10
:102130008091E80082FD7FCF8091E80080FF75CF1D
:102140009091F3008091F2002115310519F088304B
:10215000910550F041E0089709F040E08091E800D7
:102160008E778093E80061CF44914093F1003196DF
:10217000215031090196E8CF803809F084CE809152
:10218000E800877F8093E800809132028093F1001D
:1021900070CE811178CE10913602123008F073CED5
:1021A0008091E800877F8093E8001093320237D94E
:1021B0001115D9F084E08093200342E061EC81E0C6
:1021C000ABD942E261EC84E0A7D942E261EC82E063
:1021D000A3D942E260EC83E09FD980912003843050
:1021E00051F482E0809317014ECE8091E30087FD89
:1021F000E1CF81E0E0CF81E0F5CF80911901877FC9
:10220000809319018091CE03811103C082E00E9466
:1022100014058091190184FF06C08F7E80931901F7
:1022200082E00E9406058091190185FF06C08F7D1E
:102230008093190180E20E94060528CBCF92DF929D
:10224000FF920F931F93CF93DF93EC018B01F42E3A
:102250008091190182FF61C0C0905004D090510458
:10226000CC16DD0619F0209709F057C080911901AE
:102270008B7F80931901C1E081FD10C080914E04D5
:1022800090914F049801281B390BC1E080911201F5
:10229000909113012817390708F4C0E080911901C3
:1022A000C0FB81F9809319016C2FC6010E948D0833
:1022B00080915C0481FF08C0809119018061809346
:1022C000190182E00E940C0580915C0485FF08C022
:1022D0008091190180628093190180E20E940C05AF
:1022E0006C2FC601F3DBF11431F08091B30485FF4C
:1022F00002C086FF25C08091B6049091B704B5D97D
:1023000080915004909151049C013052211530432A
:1023100008F499270DDC71DF0FC0CE0190528115B2
:102320009043B0F4CE01992703DC80915004909142
:102330005104C817D90779F310934F0400934E0442
:10234000DF91CF911F910F91FF90DF90CF90089573
:10235000CE01EACFCF93DF93EC0149855A856D8595
:102360007E850E940A098B810E9414058FDA85E020
:10237000FE0111928A95E9F7DF91CF910895CF93ED
:10238000DF93EC018C8181FD10C082608C83809191
:102390005F049B81892B80935F0478DA4F81588595
:1023A0006D857E85CE010E940A0910924B04109221
:1023B0004A048C8180FD02C0CE01CCDFDF91CF9139
:1023C00008950F931F93CF93DF9308E914E0C9EDAD
:1023D000D0E0CE010E947033F80161918F0168173F
:1023E00019F0CE010E948C332196C130DC0789F7A9
:1023F000DF91CF911F910F9108950F931F93CF936A
:10240000DF9308E914E0C9EDD0E0CE010E947033FB
:10241000F80181938F012196C130DC07B1F7CAE53D
:10242000D4E0FE0185919591009711F0FC0109958A
:102430002C96F5E0C632DF07A1F7DF91CF911F910F
:102440000F910895E8E9F4E0128E138E8FEA90E080
:102450009183808385E0848F28E833E1338322836E
:1024600022E330E0378B268B28EC30E0318F208F51
:10247000158E35A324A3178E168E20E530E031A3E8
:1024800020A382A317A216A29CDF88DB1092B403BC
:102490001092B30380E084608093B40360E074E042
:1024A00084E090E00E94A633A8CF0F931F93CF93B0
:1024B000DF93962F942B982B943010F528E0629F91
:1024C000E0011124C40FD11DC40FD11D30E2839F40
:1024D000C0011124C80FD91FCE0189960E94703304
:1024E000082F10E0102F0027CE018A960E9470332B
:1024F0009801282BC901DF91CF911F910F91089569
:1025000080E090E0F8CFFF920F931F93CF93DF937B
:10251000F42E843068F5633058F524E0629FE001C2
:1025200011243CE0839FC00DD11D1124C755DF4FFE
:1025300081E084279E01280F311D280F311DC9011C
:102540000E947033082F10E0102F002781E090E0E8
:10255000F11002C083E090E08C0F9D1F0E94703349
:102560009801282BC901CDB7DEB7E5E00C94F8320D
:1025700080E090E0F8CF2091230330912403232BB7
:10258000C9F4703F39F4603FA9F480912103909120
:1025900022030895743038F4982F962B943050F419
:1025A000462F672F82CF7D3F41F4633018F441E01E
:1025B000843050F080E090E008957C3FD9F763309C
:1025C000C8F78430B8F740E09ECFA0E0B0E0EBEE73
:1025D000F2E10C94DA327C010091380580913705E4
:1025E000082BC3E0D0E010E0C8010C2E02C0959586
:1025F00087950A94E2F780FD09C02197A8F7D12CAE
:102600008D2DCDB7DEB7E7E00C94F632DC2EB701A6
:102610008C2FB1DF0E941C05019779F3F1CFCF9386
:10262000DF93D82FC92FD1DF6D2F7C2FA4DF0E941D
:102630001C05DF91CF910895FC018481811561F023
:1026400087819085009721F00E941C050C949C03C3
:1026500080819181E4DFFACF80E008951F93CF93CA
:10266000DF93182FD92F611589F0411579F0ADDF6F
:10267000C82F682F812F9D2F0E943404612F7D2F3A
:102680008C2F79DFDF91CF911F9108950E944E0426
:10269000C82FF4CFFC01462F87819085009721F445
:1026A000658180819181DACF0895382F292FCB0160
:1026B000A32FB22F8F3522E09207A105B10520F498
:1026C0008F559E4F0C94703380E0089585E290E022
:1026D0000E947033853E89F486E290E00E94703358
:1026E0008C3159F487E290E00E94703391E0873595
:1026F00009F090E0892F8170089580E0FCCFAAE076
:10270000B0E0E5E8F3E10C94D232A0901E03B09063
:102710001F0381E090E090931F0380931E0338E332
:10272000832E33E0932EC12CD12C10E0360100E033
:1027300019C021E030E0123020F4F7018591959125
:102740009C01452D602F812F4AD8539422E0E20E40
:10275000F11C34E05312EDCF0F5F84E0680E711C62
:10276000043049F0C301880F991FFC01E850FD4F68
:102770007F01512CDECF740100E021E030E0123007
:1027800020F4F701859195919C0141E0602F812F04
:102790004CD821E030E0123028F4F70132968591D0
:1027A00095919C0140E0602F812F3FD80F5FF4E0AE
:1027B000EF0EF11C033009F71F5F2CE0820E911C15
:1027C00030E1C30ED11C143009F0B0CF3BDE1A82C9
:1027D00019821C821B821E821D8218861F8288EC31
:1027E00090E09A87898701E011E0CE0101967C0193
:1027F0004AE050E0B801C7010E94AA33065F1F4FAC
:102800006701013591E0190799F78AE0F701119204
:102810008A95E9F74AE050E0B801C6010E94AA3360
:10282000065F1F4F013AF1E01F07A1F7B0921F03A7
:10283000A0921E032A96EFE00C94EE32AAE0B0E0DC
:10284000E4E2F4E10C94D932E1E9F2E080E5DF0161
:102850001D928A95E9F7E0E6F4E088E3DF011D9236
:102860008A95E9F781E9C82E82E0D82E7F0101E53B
:1028700011E0F701D182C0824AE050E0B801CE01F8
:1028800001960E94603388E0FE013196D6010190E6
:102890000D928A95E1F789859A85D70113969C93C5
:1028A0008E931297BAE0CB0ED11CE7E0EE0EF11C2E
:1028B000065F1F4F013AF1E01F07D9F62A96E8E0BC
:1028C0000C94F532282FCB01283070F44AE0249F75
:1028D00090011124B9016F5F7E4F4AE050E00E94E1
:1028E000603380E090E008958FEF9FEF0895AAE0B5
:1028F000B0E0EDE7F4E10C94DF329C0197558115CF
:10290000914068F4BE016F5F7F4F822FDBDF892B20
:1029100031F489859A852A96E2E00C94FB32809105
:10292000B0049091B104F7CFA0E0B0E0EAE9F4E19F
:102930000C94D832EC0188818115D9F0813009F0EE
:102940003FC08981813021F48A8123961CD9F3CF3D
:10295000823021F48A81239611D8EDCF833021F47F
:102960008A812396C1D8E7CF843041F02296811125
:10297000E2CFCDB7DEB7E9E00C94F4328A8123963A
:1029800020E030E09AE0682F6053770BAB016A30AB
:10299000710560F02115310551F3EFE9FFE0319742
:1029A000F1F700C0000021503109F4CF929FB0012F
:1029B000939F700D11249A01260F371F8991E3CF41
:1029C000E82FF0E0E155FE4FB490282F269526958C
:1029D000269530E0F901E156FE4FE4908770F12C26
:1029E000082E02C0F594E7940A94E2F7E0FAEE2488
:1029F000FF24E0F8F901E157FE4FC490D12C082ED6
:102A000002C0D594C7940A94E2F7C0FACC24DD241E
:102A1000C0F8F901E158FE4F049110E002C015958D
:102A200007958A95E2F701701127E114F10419F076
:102A300081EE0E94BE0CC114D10419F086EE0E94F2
:102A4000BE0C60E070E08B2D88D8C114D10411F069
:102A500086EE4AD8E114F10411F081EE45D8011553
:102A6000110511F08CE28FD8219665CFA6E0B0E079
:102A7000ECE3F5E10C94CF327C01DC0114968C91EF
:102A8000811509F41CC260E0C70104DE9C01F70156
:102A90008681803170F44091C3039091C203491341
:102AA00033C09091BE03911521F09091BF039031F6
:102AB00058F1D70115969C91911110C02115B0E5E0
:102AC0003B0708F0ABC02115E0E23E0708F0BBC0B1
:102AD000283E310590F4203E3105B0F43093B80320
:102AE0002093B703D70112968D919C919093B603D2
:102AF0008093B5031092180107C0C9019A958115FA
:102B00009F4160F72111EACF61E0C701C3DD8C016D
:102B1000F7018581811531F180914A0490914B0430
:102B2000009701F108171907E9F09C013327887F06
:102B30009927E0E0F0E0892B41F48FE0829FF001DB
:102B4000839FF00D1124EE52FC4F848184608483B6
:102B500011830083CF0113DC10925F0461E0C70191
:102B600099DD8C01D70115968C91811509F4F0C07F
:102B7000C80197578038910508F097C1003108F0D7
:102B80009EC16EE572E080E090E08FDD811197C11B
:102B9000C12CD12C7601011158C0E4E03E2E8E01EB
:102BA0000F5F1F4FD801E32D1D92EA95E9F746010B
:102BB0005701FFEF8F1A9F0AAF0ABF0AC701B6017C
:102BC00074DD8983811509F47AC1813009F0BDC0B3
:102BD0002601370122E0420E511C611C711CC50107
:102BE000B40163DD282E8A83811509F468C18FEF53
:102BF000820D833008F03DC0C301B20156DD8B83E6
:102C0000811511F0C80190DE4601570133E0830EB3
:102C1000911CA11CB11C75016401C4CF203E42E58A
:102C2000340760F4203C52E5350708F06DCFC90148
:102C300080529245809708F051CF66CFC9018757DF
:102C40009C470297F8CF8031F6CFBFE5CB16B2E0B4
:102C5000DB06E104F10409F432C1C701B60125DD48
:102C6000EFEFCE1ADE0AEE0AFE0A8111EECF015016
:102C700092CF8BEF820D833098F54601570143E0E8
:102C8000840E911CA11CB11CC301B2010EDD8B830B
:102C9000811509F4C0CFC501B40107DD8C83811112
:102CA00008C04601570154E0850E911CA11CB11CBF
:102CB000B2CF8B819C818130AFEF9A0710F0982FB3
:102CC0008827B6E02B1631F0E7E02E1631F00E948F
:102CD0006425E7CF0E942225E4CF0E944325E1CF5F
:102CE000F4E0530142012F1296CFC301B201DDDCA3
:102CF000782E4601570124E0820E911CA11CB11CC4
:102D0000C701B6016D5F7F4F8F4F9F4FCEDC7114AF
:102D100009F4D5C0811509F4D2C08150990B4FEF49
:102D2000489F9001499F300D1124472D4150550B6C
:102D3000240F351F2150310908F46DCF8FE99FE032
:102D40000197F1F700C00000F5CFC801EDDD63CFBA
:102D50000115A7E51A0708F4C4C00115B8E51B075B
:102D600008F009C66801E7E5DE1A64EC73E08C2D13
:102D7000A9DD892B29F58FE08C9DF0018D9DF00D4B
:102D80001124EE52FC4F8281813009F074C0809191
:102D9000C4039091C503892B99F08091C60390914B
:102DA000C703892B69F08091C8039091C9032091D2
:102DB000CA033091CB03822B932B892B09F465C076
:102DC0008091CE03811509F47BC1D0905C040E94F0
:102DD0009D0988579C4E9093D0038093CF03F701B1
:102DE0008581811509F46CC18D2D8D7981113CC0CF
:102DF0000115F0E51F0708F0CBC0011520E412070C
:102E000008F03FC1063E110509F4E7C0C801905221
:102E10008115904208F0D1C0D70116968C9180316F
:102E200008F421C16801DD248091190180FF35C1BA
:102E30008DEF0E941405BDE2CB16D10409F48CC1BC
:102E400008F080C1F8E2CF16D10408F028C12EE1C5
:102E5000C216D10408F028C134E0C31AD1084AE1EF
:102E6000C416D10408F478C10E94B50C8091D10336
:102E70000E94060525C1823009F0A2CF8091C803C7
:102E80009091C903892B09F49BCF2FE02C9DC001A1
:102E90002D9D900D1124FC01EA52FC4F20812E7FC4
:102EA00020838E529C4F6BDA8BCF0337FCE71F07D2
:102EB000C1F48091CE03811531F00E94B50C2696A5
:102EC000E2E10C94EB3210925C040E949D09885759
:102ED0009C4E9093D0038093CF0381E08093CE03E8
:102EE000EECF023A22E51207C1F158F4C801905220
:102EF0008115904218F1013E110579F1053E110549
:102F000003C0023B52E5150709F05ACF25EE30E029
:102F10002770332781E090E001C0880F2A95EAF7F7
:102F20002091D1033091CE033115F9F0F7013581AD
:102F30003115B1F0282B2093D103C1CFD7011696BC
:102F40008C91803108F03CCF812F99278F71992780
:102F50008230910511F04297D7CF21EE30E0D8CFE3
:102F6000809582238093D103AACF322F3823311545
:102F700009F426CF982F909592239093D1030E9425
:102F80000C05D70115968C91811509F498CF18CFAF
:102F9000003EB2E51B07C0F4003CE2E51E07E8F482
:102FA000003AF2E51F0758F4003622E51207A8F4AC
:102FB000C80192558034910580F0680135CF043BFB
:102FC00032E5130751F0F9CF09374CE7140708F041
:102FD00046C007375CE7150780F38091B30480FF94
:102FE0002AC00E949D096C01F7018581811509F4B1
:102FF0001DC18091190182FF05C040E0B60180E04B
:1030000090E01CD90431FCE71F0709F40BC105311E
:103010002CE7120709F4C2C003313CE7130709F497
:10302000F7C0C80190528115904308F0C0C01092BB
:10303000510410925004D70115969C9180915C0424
:103040008272F801911509F49BC1E052F847EB3008
:10305000F10508F0C0C1E353FC4C0C942D330B3741
:103060008CE71807AFCF812F8F71843109F4B5CF6A
:10307000863171F00E94B50C8091D1030E94060543
:10308000ACCFD70116968C91803108F0CBCEA5CF6E
:1030900056EEC52E52E1D52EC7CE8FEFCACE5AE2DC
:1030A000C516D10409F0E0CE8091D103811531F02D
:1030B00080915F0492E0892780935F040E94460C10
:1030C000C80197558115914008F087CF5801B8EF96
:1030D000AB22BB24A114B10409F0F1CE2FE0029F72
:1030E000F0011124AF014E525C4F6A01D7011596D1
:1030F0008C91EA52FC4F908180FB90F9908381156E
:1031000089F10E949D0990934D0480934C04F6012F
:1031100082818F5F828380915F0490915C04892B10
:1031200083834581568165857685C6010E940A099B
:10313000D60114968C9181FF5801B0924B04A09255
:103140004A044BCF8CE4C816D10409F4ADCF9DE2FC
:10315000C91692E0D906A6CF80915F048260809361
:103160005F04A2CFFA014385548565857685C60143
:103170000E940A09D60114968C9181FF2ECFC601B8
:10318000E9D880914A0490914B040817190709F077
:1031900024CF10924B0410924A041FCF9091190132
:1031A000892F8E7F90FF81608093190126D88091AE
:1031B000190180FF40CF0832110508F04DC00E31D3
:1031C000110508F05AC0C80104974A9730F580915C
:1031D000B30484FD22C0D70115968C91811509F4A2
:1031E000ADC080915C048D7F811509F44BC01092B5
:1031F0005104109250048091B30481FD43C060E0FB
:10320000C8010E948D0860E0C8010E94660D57CE7B
:1032100080911901816080931901F70185818111E5
:1032200006CF09CF809119018E7FBECF8091190101
:103230008F7E013E110531F0053E110531F480917C
:1032400019018F7D80931901B2CFC8019052811569
:10325000904308F0ACCFEFCE0933110558F40D328E
:10326000110518F40B321105C1F68091B30482FDEB
:10327000D4CFB1CF04361105F7CF8091B30483FDCD
:10328000CCCFA9CF89E0F701A2E5B4E001900D927F
:103290008A95E1F7109255041092540480915004DD
:1032A0009091510408171907B1F52091B30425FF37
:1032B00032C03091190131FF02C026FF2CC020918D
:1032C0004E0430914F047601E21AF30A10DBE8163F
:1032D000F90608F580915C0481FF08C0809119010E
:1032E00080618093190182E00E940C0580915C044A
:1032F00085FF08C08091190180628093190180E2E6
:103300000E940C05609119016695617080915004CE
:10331000909151047ACF80915C04109351040093F2
:103320005004D0924F04C0924E04827084609091F9
:103330001901997F892B80931901C1CD40E0B60115
:10334000C8010E941E11BBCD0E94D106B8CD8115C7
:1033500059F10E941B07B3CD811559F10E943C071A
:10336000AECD811559F10E945107A9CD811559F1B2
:103370000E946907A4CD811559F10E947F079FCD56
:10338000E054F847ED30F10530F5E852FC4C0C9470
:103390002D330E94DB0681E00E94C90690CD0E9479
:1033A000E906F9CF8115A9F20E94110788CD811590
:1033B000A9F20E94330783CD8115A9F20E94450727
:1033C0007ECD8115A9F20E945D0779CD8115A9F204
:1033D0000E94750774CD0737BCE71B07F9F0083763
:1033E000ECE71E0749F19801205E32452032310595
:1033F00028F5911123C00F7181E090E09C0102C07B
:10340000220F331F0A95E2F78901622F83E090E0D3
:103410000E948C33802F0E94C00351CD81E0911512
:1034200019F00E94C60302C00E94D00343E062E08C
:1034300081E00E94670443CD82E0F1CF80915B047C
:10344000B09038052B2D30E02095309550E02823A2
:103450003523232B19F08B2180935B040B373CE73A
:10346000130749F4911509F42ACD8B2D0E94890385
:103470000E94F00824CD003442E5140708F04FC044
:10348000003252E5150708F051C0011580E5180714
:1034900018F50115A0E41A0708F05EC0911509F4AB
:1034A00073C00130FCE71F0709F4B4C003302CE7F8
:1034B000120709F4A9C001151C4709F065C00E9454
:1034C000CE0D4FEF54E38CE0415050408040E1F787
:1034D00000C000000E94690B980130552115324050
:1034E000E8F6980145E0369527954A95E1F7822F51
:1034F0008F7020915B0430E041E050E0082E02C064
:10350000440F551F0A94E2F724233523232B31F26D
:103510009111AECF10925C040E94460CD0CC980161
:10352000205C32452032310508F0B8CF802F8F71F2
:1035300020915B0430E041E050E0082E02C0440FCF
:10354000551F0A94E2F724233523232B09F4A6CF31
:10355000911509F4B4CC8CCFF7018681803108F045
:103560009DCF911111C0812F8F7021E030E002C0FA
:10357000220F331F8A95E2F740915B0450E0242329
:103580003523232B09F09BCCD70117962D913C9125
:103590002115310509F440C0C9010E941C05182FEE
:1035A000092F86E0F701DE01119601900D928A95B0
:1035B000E1F7D7011596DC9015971696CC90C2943A
:1035C0009FE0C922802F82958F70883009F4D2C085
:1035D00008F04EC08430B8F5823008F459C0802F0E
:1035E0008F70902F907F903211F08295807F1130F4
:1035F00009F08BC09091BA04D11409F480C09C15D5
:1036000028F10E949D0C22C06FEF7FEF80E090E0D8
:103610000E94A6330E94EC0DF701C080D180911565
:1036200069F0C6010E94E512182F682FC6010E949A
:103630003404B601812F0E94BB12AFCFC6010E9495
:103640004E04182FF6CF843009F477C0812F902FC5
:103650000E949C03811541F0D11409F461C1C11489
:1036600009F455C110923B0560E0C70113D827CC7F
:10367000893009F4ECC08A5F8F70823038F7123FCE
:1036800009F0F8C0802F8F71D11409F425C1EFC063
:10369000B02FBF70BB2E003118F0B29480EFB8226B
:1036A000D114B9F0B11459F080E2810F883010F0D4
:1036B000111109C08B2D0E9406050E94460C812F16
:1036C0000E94BE0CC3CF80915F048B2980935F045E
:1036D000F4CF812F0E94740DB11409F4B7CF80E2AA
:1036E000810F883010F0111106C08B2D0E940C053F
:1036F0000E94460CABCF8B2D0E941405F9CFC91642
:1037000008F0A4CF0E94AB0CA1CFD11421F0C114BA
:1037100009F477CFD4CFC114A9F38091B804909164
:10372000B904193321F08091B6049091B7040E9436
:10373000350B812F0E94740D89CF802F8695869539
:103740008370811569F0813009F080CF812F902F2F
:103750009370D11002C080E090E00E94460976CFBD
:10376000812F902F9370D11002C080E090E00E94D2
:103770001E096CCF802F8370811135C0D11028C0F5
:10378000412F429546954770440F440F812F8F700B
:10379000042E01C0880F0A94EAF7212F207114FF2C
:1037A00007C02FE030E001C0220F4A95EAF72095CC
:1037B000302F369536953370323081F0333061F0EA
:1037C00040913705313039F0822B84230E94C003A9
:1037D0000E940F093BCF842B822BF8CF822B909134
:1037E00037058927F3CFD11449F100FFF1CF412FDD
:1037F000429546954770440F440F812F8F70042ED9
:1038000001C0880F0A94EAF7212F207114FF07C026
:103810002FE030E001C0220F4A95EAF72095302FC3
:10382000369536953370323079F0333059F0313087
:1038300041F0822B8B210E94C303CACF823040F219
:10384000D6CF8B29822BF7CF822B8B25F4CFE02F7D
:10385000EF70BE2ED11439F08E2F0E94C603812F37
:103860000E949D0CB5CF812F0E94AB0C8B2D0E9426
:10387000D003AECF60F4103FB9F0113F49F1D1143D
:1038800089F1C11461F1812F0E94BE0CA1CF133FB9
:10389000B1F780E0D11479F281E0902F9F7101C0DF
:1038A000880F9A95EAF7C7CF8091BA04D11461F0D6
:1038B000C81608F08DCF202F2F7181E090E001C055
:1038C000880F2A95EAF7C1CF8C1508F481CFF3CF82
:1038D000802F8F71D11459F20E94C60379CF802FA7
:1038E0008F71FACFC11481F08091B8049091B9041E
:1038F000193321F08091B6049091B7040E94350BE2
:10390000812F0E94740D64CF802F8F71B0CF809172
:103910005E0480935D0480915C0480935E04A4CE79
:1039200040E060E089819A810E942E139C01009101
:103930005C04C11429F010923B0500935E0494CE00
:103940008091390590913A0528173907B1F7809190
:10395000B50482FFF0CF80913B05811561F3809122
:103960005D040E949D0C812F0E94C30D80915D0417
:103970000E94AB0CE0CF0337FCE71F0706CBA0E0AB
:10398000B0E0E5ECFCE10C94DA328091BF038031C9
:1039900008F048C08091BE03811509F443C0C0916E
:1039A000C30389E0D82E8091C2038C17D9F1EC2E85
:1039B000F12CDC9EE0011124FE01EE59FC4F8481C4
:1039C0008115A9F191818091BA03981330C090813B
:1039D0008091B90398132BC08581811128C0028181
:1039E00013818091BB039091BC03081B190B60E00D
:1039F00089EB93E00E944A130E9477140817190775
:103A0000B0F48091BF038F7080618093BF03C85969
:103A1000DC4F88818F708061888389EB93E026D8A2
:103A20000E94FC04CDB7DEB7E7E00C94F632E70164
:103A30002196C770B8CFCF92DF92FF920F931F935A
:103A4000CF93DF93182F092F89E0F82EC091C3037D
:103A50008091C203C81799F1FC9EE0011124CE01A8
:103A60008E599C4F6C01FC018581811589F0C6013E
:103A70000E941C13811561F0FE01E859FC4F208162
:103A80002F7020612083F601808191810E94010EB8
:103A9000C6010E9436152091C30330E02F5F3F4FCF
:103AA000277033272093C303CE59DC4F89818013BD
:103AB000CDCF88818113CACF8D81811539F2DF91F5
:103AC000CF911F910F91FF90DF90CF900895EF92CB
:103AD000FF921F93CF93DF93EC01209118012115E2
:103AE00041F010E0812FDF91CF911F91FF90EF9077
:103AF0000895EA80FB80E61AF70A24EFE21621E037
:103B0000F20678F760E0CE010E944A139C01305221
:103B10002115304330F70E94C704811511F38091BD
:103B2000B7039091B8030E94C704182F8115C9F2FA
:103B30008091BE049091BF04853F21E0920710F070
:103B400084EF91E0E816F90660F68E818F7080614F
:103B50008E83888199810E94010E0E948604CE0185
:103B60000E943615BFCFAFE0B0E0E9EBFDE10C9469
:103B7000D0328C0186E0F801DE011A9601900D9298
:103B80008A95E1F7D8014C9011963C9011971296C6
:103B9000ED90FC90139714965C90149715966C908A
:103BA00061100CC050916103252F30E0E0E08E2FB2
:103BB0000E2E000C990B821793073CF159EBA52EA2
:103BC00053E0B52E8091BD03811151C05114D1F045
:103BD000611409F43FC3C8010E941C13811509F444
:103BE00039C36091B5037091B603C80170DF8111CC
:103BF00009C089E0F801A9EBB3E001900D928A9524
:103C0000E1F7BDDEFF24F39497C0880F991F8F5A08
:103C10009C4FDC0111964C911197431103C08C917C
:103C2000481611F0EF5FC3CFEF3F41F2D80116966F
:103C30008C9116978F70806116968C93E517A0F47F
:103C4000AFEFA50FA0936103EA1770F4F0E0EE0F59
:103C5000FF1FEF5AFC4FB0E0AA0FBB1FAF5ABC4F7B
:103C60008D919C91918380830E948604A7CF60E010
:103C700089EB93E00E944A136C017090BE0380911F
:103C8000BB039091BC034701881A990A60E089EB55
:103C900093E0711409F479C20E944A130E947714C8
:103CA0008816990608F026C2511409F4ABCF80910A
:103CB000BA03F8019181B090BF03F0E1BF1608F09C
:103CC000D3C198135BC09091B903D8018C9198131C
:103CD00055C02091C0033091C10317968D919C91DE
:103CE0002817390709F04AC0611048C08B2D8F7022
:103CF00080618093BF0389EB93E00E943615809129
:103D0000BF03F8018683F090BB03E090BC0349E059
:103D1000D42E0091C3038091C203081751F0D09EA6
:103D2000800111240E591C4FD80115968C918111D8
:103D300008C00E94FC04F12C8F2D2F96E1E10C9419
:103D4000EC32F801B280C380C8010E941C138111BB
:103D50000EC0C8010E9436158091C30390E0019601
:103D6000877099278093C303FB2CEC2CD2CF6F2D47
:103D70007E2DC801ACDE8111EFCFDBCFF0E2DF1A80
:103D8000C11420E3D20608F084C0611005C140E0F0
:103D9000632D842D0E94160B81114FC040E0632DCE
:103DA000842D0E94160BF82E811509F429C18091EB
:103DB000B50480FFC0CF89EB93E00E94361560E028
:103DC00089EB93E00E944A138C01F090C3037F2C8F
:103DD00098E0E92E29EB822E23E0922E39E0432E43
:103DE0008091C2037816A1F0A72CB12C479CC0018A
:103DF0001124FC01EE59FC4F6F0160E0CF010E94DD
:103E00004A13582E692ED60115968C91811197C0B0
:103E1000B8E0EB1618F419E0EF10ACC08A859B856A
:103E20000ADE0E9486040E94FC0489E0E9EBF3E0CC
:103E3000DF011D928A95E9F77ECF60E0C8010E94FC
:103E40004A138091B50483FFA9CFB80189EB93E0B1
:103E50000E9493048111A2CF8091BF038F70806173
:103E60008093BF038091B9039091BA030E94010E21
:103E700089EB93E00E943615E9EBF3E089E0DF017E
:103E80001D928A95E9F78A859B85D5DD0E94860477
:103E900050CF611409F482CF8091BF038160809379
:103EA000BF038091B50481FF46CF89EB93E00E9468
:103EB00036150091C3038091C203081709F4CCC0E2
:103EC000E02EF12CB9E00B9FC0011124FC01EE594A
:103ED000FC4F6F01CF010E941C13811509F4BCC077
:103EE00089E0F601A9EBB3E001900D928A95E1F724
:103EF000C701019687709927082F8093C3030E94FA
:103F0000FC0489E0F82E8091C203801709F411CFD8
:103F1000F09E800111240E591C4FC8010E941C13F1
:103F2000811107CFC8010E9436158091C30390E02C
:103F3000019687709927082F8093C303E4CF10520E
:103F40000115E0E31E0708F063CF8091B50483FDFF
:103F50000AC0E72CC5010196F82FF7707F2E052DBA
:103F6000162D46013DCFB601C4010E949304811570
:103F700089F3EFCF1F9DC00111248E599C4F0E94E1
:103F800036152091C30330E02F5F3F4F2770332752
:103F9000F22E2093C30340CF8091BF0381608093B2
:103FA000BF0360E0C8010E944A138091B50483FFFB
:103FB00078CFB80189EB93E00E949304811171CF0F
:103FC000F090BF03E894F0F8F092BF03C8010E949C
:103FD0001C138111B0CE8F2D8F7080618093BF0331
:103FE0008091B9039091BA030E94010E0E94860449
:103FF00089EB93E00E943615E9EBF3E089E018CFF6
:104000008A859B850E940F13292F22952F7090344B
:1040100050F49F70223080F0911599F0F80196814C
:10402000903178F489CE2A5F2F70223078F0C80161
:104030000E943615F72C80CE911519F0811509F4E0
:104040007BCE805E883008F477CEF1CF803F08F4D5
:1040500073CE815F8330F7CF89E0E9EBF3E0DF01D6
:104060001D928A95E9F74DCF98131EC09091B90320
:10407000F8018081981318C02091C0033091C103CA
:10408000878190852817390779F461100DC0B682B1
:10409000C8010E94361589E0F801A9EBB3E0019050
:1040A0000D928A95E1F7AECDC8010E941C138115CF
:1040B00009F4D0C0611409F4CDC08091BF038032EF
:1040C00008F497CD8091B9039091BA039A838983BC
:1040D000FC82EB828091BD038D831E82BF82809122
:1040E000C0039091C10399878887CE0101960E94F1
:1040F00036157FCDD090BF03F0E1DF1638F489EBA1
:1041000093E00E94361589E0D50193CE511409F44D
:1041100079CD9091BA03F801818198131AC09091DA
:10412000B9038081981315C02091C0033091C10359
:10413000878190852817390761F461100AC0D682FB
:10414000C8010E94361589E0D5011D928A95E9F7CC
:1041500059CDC8010E941C13811509F47BC061145C
:1041600009F478C08091BF03803208F442CD809179
:10417000B9039091BA039A838983FC82EB82809180
:10418000BD038D831E82DF82AACF0E944A130E9444
:1041900077148816990608F061C0511409F432CDDD
:1041A000611409F457C09091BA03F8018181981302
:1041B00039C09091B9038081981334C02091C00315
:1041C0003091C103878190852817390759F580916F
:1041D000BB039091BC03E81AF90A60E089EB93E015
:1041E0000E944A138091BC049091BD04E816F90620
:1041F00008F051CF8091BF0380FD4DCF803108F48E
:104200004ACFD80116968C931697982F907F903F9F
:1042100009F43ECF982F907F905F8F70892B169670
:104220008C9336CFC8010E941C13811571F06091E8
:10423000B5037091B603C8014ADC811509F4D9CCE5
:1042400089E0E9EBF3E0DF0180CF8091BF0381607B
:104250008093BF03C8010E943615D4CC89E0F501D4
:1042600011928A95E9F767CDA2E1B0E0EAE3F1E2C5
:104270000C94DB320A871B872C873D874E875F872C
:10428000688B798B8A8BCE010A966DDC0C851D8537
:10429000FE84811127C02091C2033091C30389E0BD
:1042A000FE013A96DE01119601900D928A95E1F792
:1042B000F114C1F0822F90E001968770992738178A
:1042C0001906B9F199E0929FD0011124AE59BC4F63
:1042D000FE01319601900D929A95E1F78093C20309
:1042E0000E94FC0489E0E82E8091C3039091C203F0
:1042F000891741F0E89EC00111248E599C4F33DC90
:10430000811125C0F11011C08091180181110DC0DB
:104310008091B5039091B603081B190B0F3FBFE3C3
:104320001B0718F081E0809318016296E6E00C9478
:10433000F7320E94CE0D1092C2031092C30389E09F
:10434000E9EBF3E0DF011D928A95E9F7CBCF80918D
:10435000C30390E00196877099278093C303C4CF6D
:10436000EF92FF920F931F93CF93DF9380913405C9
:10437000E0914C02CDE0811139C0CDB7DEB7E6E067
:104380000C94F732D1E0DE0FD0934C02EE2EF12CDC
:10439000CE9FF0011124E453FB4F8481811529F154
:1043A00087819085892B21F481859285019651F42E
:1043B0000081118122813381448155816681778119
:1043C000808552DFCE9DF001CF9DF00D1124E45386
:1043D000FB4F14828091CE03811521F08091190149
:1043E00080FD0DC08FEF0E941405ED2F80913405E4
:1043F000E81740F21092340510924C02BECF8DEFB8
:10440000F2CFA4E0B0E0E7E0F2E20C94D0322091E9
:10441000CB04298397E0992E01E010E02DE0322EA5
:1044200034E0532E882483948091CA04998189139F
:1044300007C096DF0E94B3082496E1E10C94EC32A9
:104440009981892F90E09C838B83FC01EE0FFF1FE5
:10445000E054FB4F80819181989ED001999EB00DD0
:104460001124FD01E05AFB4FFA83E98324812111D5
:104470005BC060903405ECECF4E060E070E0712C1F
:10448000661508F04FC0A384B484A981BA81CD9089
:10449000DC902FEF3FEF412C442D50E07601E40CEF
:1044A000F11CE40CF11CD701ED90FC90E114F10437
:1044B00039F0AE14BF0409F0A90143949A01ECCF7E
:1044C0002F3F3207D1F1D80102C0AA0FBB1F2A9596
:1044D000E2F77A2A9801042C02C0220F331F0A94B3
:1044E000E2F7A901415051097416150629F5369EC7
:1044F000F001379EF00D1124E453FB4F989ED0013C
:10450000999EB00D1124A05ABB4F12962D913C914B
:104510001397308727835482108211829287818774
:1045200015968C920E94C4088B819C8101969A8377
:1045300089838370898378CF14826F5F7F4F3D9624
:104540009FCF109236051092350510921A01809176
:10455000CA048093CB040E94B30802CF2F923F92EB
:104560005F926F927F928F929F92AF92BF92CF9203
:10457000DF92EF92FF920F931F93CF93DF93CDB70C
:10458000DEB76C970FB6F894DEBF0FBECDBF4B8B76
:104590005C8B6D8B7E8B8F8B692F988F192F81157C
:1045A00009F44FC040E08B899C890E942E139C0126
:1045B000111549F010923B0590933A058093390507
:1045C00010925F040AC08091390590913A058217D4
:1045D000930719F481E080933B05188A198A1A8A97
:1045E00086E0FE017396DE011A9601900D928A957F
:1045F000E1F78E858115D1F061E0CE010A960E9427
:104600004A1361E0CE010A960E944A1361E0CE018E
:104610000A960E944A135C0180352CE79207A1F4A8
:104620008F85811529F181E080931A010A851B8508
:104630002C853D854E855F85688979898A8914DE58
:10464000D2C0911551F2BCCF81354CE7940729F4C3
:104650008F85811569F075DFE9CF82359C4741F47C
:104660008F85811529F080911A018111F4CFDBCF5C
:1046700020E6E22E24E0F22E712C812C912C6F8406
:10468000D7016D917C91CC24CA94DD24DA9480E02A
:10469000282F30E0FB01E80FF11DE80FF11D4081EC
:1046A00051814115510539F0A416B50609F096015E
:1046B0008F5F6901EDCFBFEFCB16DB0609F48AC12E
:1046C000F701448150901A014111512CD7011596E0
:1046D0003C90159716962C911697611409F41BC1FE
:1046E000511409F418C10091AE041091AF043110B7
:1046F00014C041E050E001C0440FCA94EAF7242BF3
:1047000016962C932091C8043091C90420173107C4
:1047100020F41093C9040093C80421E030E0F901AB
:1047200002C0EE0FFF1F8A95E2F7CF010197D70174
:1047300016962C912817190609F0D2C0C09035059D
:10474000D0903605C114D10409F465C00E949D09BA
:104750008C199D090817190708F05DC081E0F70161
:104760008483782ABFEF8B1A9B0AE7E0EE0EF11CD8
:10477000F8E08F16910409F082CF611409F42CC17E
:10478000711409F429C10E949D0990933605809304
:10479000350580913405883030F591E0980F90937D
:1047A000340599E0FE013A96DE01119601900D92D2
:1047B0009A95E1F72DE0829FC001112484539B4F0D
:1047C00029E0FE013196DC0101900D922A95E1F776
:1047D0002FEF3FEFDC011A963C932E9319971C960E
:1047E000BC92AE921B976C960FB6F894DEBF0FBECC
:1047F000CDBFDF91CF911F910F91FF90EF90DF9090
:10480000CF90BF90AF909F908F907F906F905F9070
:104810003F902F9008954091CB042091CA04342FEB
:1048200080E090E057E0A1E0421709F446C0242E52
:10483000312CF101EE0FFF1FE054FB4F008111817D
:10484000509FF001519FF00D1124E05AFB4F608101
:1048500071817C8F6B8FC12CB0E0D12CEB8DFC8DE6
:10486000ED0DF11DED0DF11D808191810097E1F0BD
:10487000F7010190F081E02DFA8FE98FB0E007C0D9
:10488000E1E08617970709F0E0E0CE2ABF5FE98DE7
:10489000FA8DEB0FF11DEB0FF11D60817181611538
:1048A000710571F7D394DACFC11491F1BD15D0F42D
:1048B00081E0D70114968C93C7013093CB048E15F9
:1048C0009F0571F030E0F901EE0FFF1FE054FB4F40
:1048D000918280822F5F3F4F237033272093CA0439
:1048E000852D3FCF509FC001519F900D1124805ABC
:1048F0009B4FFC01A4838E159F05F1F2431302C068
:104900003F5F3370B1016F5F7F4F462F43708CCF95
:1049100080E090E0F7CF30E0311024C061E070E03B
:1049200002C0660F771F8A95E2F7CB01019728171F
:10493000390791F0512CE1E0F0E002C0EE0FFF1FCB
:10494000CA94E2F76F01C094D70116968C9116971E
:104950008C2116968C93C4CF411569F3C4010E9433
:10496000C408E8CFA9010C2C02C0559547950A94BC
:10497000E2F7C901019782239323892B39F540FF80
:1049800025C0D70112968D919C91892BD1F087E09B
:10499000FE013196DF011D928A95E9F70E949D097B
:1049A0009C018B839C8384E08D83F70192818381BA
:1049B000792F9887898709811A8144E05E816F8108
:1049C00053DCD70115961C92532CB5CFB42FB17080
:1049D0005B2EB1CF80E0C5CE9091CB048091CA040C
:1049E000981731F00EDDB1E07B1609F4FCCE1ECE37
:1049F000B7DC10923605109235050E94B308F3CF4C
:104A0000A6E0B0E0E6E0F5E20C94DD320E949D09FC
:104A10008C0180912503909126038017910771F0F6
:104A200019821A820E949D09BC0149815A8180E045
:104A300090E094DD10932603009325032696E4E08E
:104A40000C94F932A6E0B0E0E8E2F5E20C94DF3233
:104A50009093220380932103811520E2920730F482
:104A60000E94510D2696E2E00C94FB3280EF898380
:104A70008A830E949D098160BC0149815A8181E03D
:104A800091E06CDDEFCFA6E0B0E0E9E4F5E20C9454
:104A9000DF329093220380932103811520E2920755
:104AA00030F40E94980D2696E2E00C94FB3280EFE1
:104AB00089838A830E949D098160BC0149815A8152
:104AC00081E090E04BDDEFCFCF93DF93D82FC92F5C
:104AD000B9DF8091B6049091B7040E94350B8D2FF9
:104AE0009C2FD1DFDF91CF9108950F931F93CF9328
:104AF000DF938C01862F64EC73E00E946214892B93
:104B000091F4C091C403D091C503209761F0F801DE
:104B10008281833039F4CE01D7DFCE01D5DFCE01DB
:104B2000D3DF01C0E0F7DF91CF911F910F9108957E
:104B30000F931F93CF93DF938C01EB0164EC73E031
:104B40008C2F0E946214892B09F057C0FE01FF27A9
:104B5000D80112968C911297EF51FD4F8130A9F434
:104B600014968C9182FD4EC080FF4CC082E0808301
:104B70008091C6039091C7030097B9F48091C40354
:104B80009091C5030097C9F110C08230A1F5149629
:104B90008C9182FD26C080FD0AC083E080838091D5
:104BA000C8039091C9030097F1F04CDF26C084E060
:104BB00080838091CA039091CB030097B1F78091D5
:104BC000C4039091C503009701F17EDF8091C60375
:104BD0009091C703009749F78091C4039091C50352
:104BE000E4CF85E080838091C4039091C503009752
:104BF00021F06ADFF1CF86E08083DF91CF911F91B2
:104C00000F91089581E08083B9CF8091C603909180
:104C1000C703B8CF0F931F93CF93DF938C01EB01A2
:104C200064EC73E08C2F0E946214892BA1F48091B4
:104C3000B6049091B7040E94350BDD27CF51DD4FAC
:104C40008881F801128218828330E9F048F48130BB
:104C500059F0823081F0DF91CF911F910F9108952B
:104C60008430B1F08530B9F78091C4039091C503C9
:104C7000009789F306C08091C6039091C7030097FF
:104C800099F301DFE8CF8091C8039091C903F7CF72
:104C90008091CA039091CB03009799F72091C403A8
:104CA0003091C5038091C6039091C703211531054A
:104CB000F9F2009731F7C901E4CF48E050E067E12D
:104CC00070E082E193E00E947D331092F502089536
:104CD000E2E1F3E089E0808380911B0190911C0167
:104CE000A0911D0181839283A3838FE784838FEF3B
:104CF0008583E3CFA0E0B0E0E0E8F6E20C94D9329F
:104D00000E94A9096093E9027093EA028093EB0282
:104D10009093EC0220911203122F1370111519F0C9
:104D2000122F1695169530910501323009F4CDC039
:104D300080F4311116C0109200016093ED0270935F
:104D4000EE028093EF029093F00281E080930501E0
:104D500003C0333009F4C1C0CDB7DEB7E8E00C942E
:104D6000F5328091040118132AC023704091030189
:104D700050E081E02417150609F480E080930201D9
:104D80008091170390910101981739F080930101E8
:104D900040E060E080E00E94CF06113091F01230D8
:104DA00009F44FC0111109C080910201811529F049
:104DB00040E060E080E00E94CF0680E01FC081E01C
:104DC000DDCF80910001C82FCC0FC80F03E00C0F7E
:104DD000C02E0D3010F09CE0C92E6091130370912D
:104DE0001403809115030E941906F62EE72ED82E83
:104DF000D0E0CC15A8F081E00C30F8F690910001DD
:104E00009F5F909300018111A7CF82E080930501FD
:104E1000809102018111A0CF11119ECF83E096CF26
:104E2000FE01E45CFE4F80A590910101892381156C
:104E300031F02D2D4E2D6F2DCE010E946A08219646
:104E4000D8CF80910001C82FCC0FC80F03E00C0F02
:104E5000E02E0D3010F08CE0E82E309116033695E0
:104E6000369521E0320F08F43FEF4091ED0250916A
:104E7000EE0280E090E0439F040E811D539F800D61
:104E8000911D1124850F911DF82ED0E0CE1508F04C
:104E9000B2CFFE01E45CFE4F80A590910101892311
:104EA000811589F0609113037091140380911503AB
:104EB0002F2D4C2F0E94A0060E941906472F282F45
:104EC000CE010E946A082196E1CF1093040123705D
:104ED000209303010E94430BA1CF8091F502811121
:104EE000ECDEC090ED02D090EE02E090EF02F09088
:104EF000F0020E94A9096C197D098E099F09603191
:104F000071058105910508F427CF1092050124CF82
:104F1000A0E1B0E0EEE8F7E20C94D132FE01319668
:104F200080E1DF011D928A95E9F706E210E091EA3F
:104F3000A92EBB24B3942FE5422E22E0522E612CE1
:104F4000712C4F0173016201B1E14B1651046104F0
:104F500071041CF080E1C82ED12CA601B501C4015A
:104F60000E947D33AC0CBD1C0D2C000CEE08FF081C
:104F70004C185D086E087F080150104019F76096C4
:104F8000E0E10C94ED326FEF85E290E00E948C330B
:104F90006FEF86E290E00E948C336FEF87E290E043
:104FA0000E948C3360E088E290E00E948C330E9483
:104FB0007F13AEDF65EE85E290E00E948C336CE1FA
:104FC00086E290E00E948C3367E587E290E00C94E3
:104FD0008C339C01CB01BA01F9013296E4914E2F3A
:104FE00050E06E17710548F0F9013496659175919E
:104FF0000E94503380E090E008958FEF9FEF089576
:10500000A4E0B0E0E6E0F8E20C94DC328B01FC01B5
:105010003396F49019821A821B821C82452B31F43C
:105020008FEF9FEF2496E5E00C94F83244E050E0D7
:10503000BE016F5F7F4FCDDF019691F381E090E07D
:105040000F2C02C0880F991F0A94E2F7092E000C5A
:10505000AA0BBB0B49815A816B817C8184239523E8
:10506000A623B72321E0892B8A2B8B2B09F420E080
:10507000F801208380E090E0D5CF9C01CA01F901BE
:105080003296E4914E2F50E08E17910558F0F901B9
:105090003496859195910E9450330E94E11180E0F1
:1050A00090E008958FEF9FEF0895A4E0B0E0EBE566
:1050B000F8E20C94D8327C016B01CA01F7013396F7
:1050C000B49019821A821B821C82892B31F48FEFD3
:1050D0009FEF2496E9E00C94F43244E050E0BE01E6
:1050E0006F5F7F4FC70175DF019689F381E090E024
:1050F0000B2C02C0880F991F0A94E2F780959095B7
:10510000092E000CAA0BBB0B49815A816B817C8153
:1051100084239523A623B723F6012081022F017053
:1051200010E00B2C02C0000F111F0A94E2F7012EB1
:10513000000C220B330B802B912BA22BB32B8983DA
:105140009A83AB83BC8344E050E0BE016F5F7F4F26
:10515000C70193DFBECFA4E0B0E0E1EBF8E20C942E
:10516000D432FE01319684E0DF011D928A95E9F781
:1051700088E7A82E81E0B82E0CE711E099249394DB
:105180007E2E8F2EEE24E394F12C20E8C22E21E017
:10519000D22EF50181915F018F3F09F446C0F8944A
:1051A000E82FE295EF70F0E021A18F70A70102C017
:1051B000440F551F8A95E2F7CA01922F982B91A3AD
:1051C00092A18095892382A3789400C0ACE7B1E0D6
:1051D000672D782D492D40959D91FB018191BF014F
:1051E0009F3F09F44AC0292F22952F70205E30E09E
:1051F000F901208130E09F7002C0359527959A957E
:10520000E2F720FD3AC089299B0121503109F901BB
:105210008083CA16DB0601F7F50182918F3F11F0FA
:105220000E940006F0EAFA95F1F7990C0A151B05A1
:1052300009F0AFCF44E050E0672D782D81EF92E088
:105240000E944333892BD9F089819A81AB81BC813B
:105250008093F1029093F202A093F302B093F402D0
:1052600081E0809330020E949D0990932F028093E9
:105270002E022496EDE00C94F0328423C5CF809169
:1052800030028115B1F300912E0210912F020E947D
:105290009D09801B910B059760F344E050E061EF9E
:1052A00072E08AE193E00E944333892B81F0809180
:1052B000F1029091F202A091F302B091F402809376
:1052C0001A0390931B03A0931C03B0931D03109229
:1052D0003002CFCFCDB7DEB7E8970FB6F894DEBF78
:1052E0000FBECDBF85B7806885BF85B7806885BF95
:1052F00084B7877F84BF0FB6F894A895809160002B
:10530000886180936000109260000FBE80E890E09A
:105310000FB6F89480936100909361000FBE81E016
:10532000809317018EEF95E090930502809304021D
:105330000E9496070E941E140E94FD110E945F0A9F
:105340000E94BC0A8091E20084608093E20078941D
:1053500080912003811599F08091E9001091EC0073
:105360008F70179511271795182B1092E9008091CF
:10537000E80083FD0E943A0E1F701093E90082E05E
:1053800084BD93E095BD9AEF97BD80936E000E9417
:105390006613811101C0F7DDE4E0F3E088E0DF018E
:1053A0001D928A95E9F783E08093030310E060E0A3
:1053B000812F0E94280861E0812F0E9428081F5F2A
:1053C0001330A9F7EFE8F1E03197F1F700C00000E2
:1053D00010E080910303181708F480C084E90E944C
:1053E000000687E90E94000684E30E94000685E328
:1053F0000E94000687E60E94000686E60E940006DC
:1054000086E90E94000684EF0E94000684E0EAE13B
:10541000F3E0DF01282F1D922A95E9F7E1EFF2E092
:10542000DF011D928A95E9F780E090E00E947833D1
:10543000833E9E4F21F40E94661381112AC063EEC1
:105440007EEF80E090E00E94A63360E082E090E092
:105450000E948C3381E08093370561E083E090E027
:105460000E948C3360E074E184E090E00E94A633F7
:105470002FDC89DD40E050E0BA018FE090E00E942F
:105480009E3340E050E0BA0183E190E00E949E33F9
:1054900014DC82E090E00E9470338093F80284E094
:1054A00090E00E9478339093B4038093B30353DE6B
:1054B000EFEFF6E721E0E150F0402040E1F700C0D7
:1054C000000049DE80911A0380FF1AC06FEF7FEF62
:1054D00080E090E00E94A6330E94690B60E0812F7B
:1054E0000E944B08082F61E0812F0E944B08E12F9A
:1054F000F0E0E050FD4F880F802B80831F5F69CF65
:1055000083E090E00E9470330E94C0030E9468080C
:1055100081E08093F50248E050E067E170E082E1CD
:1055200093E00E9460331092F50280911203843060
:1055300008F4CEDB86E091E0909348038093470324
:105540008091200310E4853009F47BC004DE09EF6C
:1055500012E0EAE1EE2EE3E0FE2ED701F801919190
:105560008D912DEF32E02E173F0709F474C0981784
:10557000B1F3D12CD701CD907D01F80191908F012D
:105580009C1429F19C24B12CAA24A394892D8A214E
:105590008115B1F0B982DA820E949D099C838B83C8
:1055A000F1E0FD8391E08C2D8A21811101C090E012
:1055B0009E8349815A816B817C818D810E94AE22BC
:1055C000B394AA0C24E0B212E1CFF801C292D394B2
:1055D00034E0D312CFCF0E94A90940C080912003AC
:1055E000843021F187DB1092F60288E190E00FB65B
:1055F000F894A895809360000FBE1093600083B765
:10560000817F846083BF83B7816083BF78948895EE
:1056100083B78E7F83BF0FB6F894A8958091600002
:10562000886180936000109260000FBE94DDEAE113
:10563000F3E081918111EAC5AEE1B3E0AE17BF0797
:10564000C1F780912003853009F4C8CF0E94CE0DA8
:105650000E940F097BCF98138CCFD2D9E0904A04D7
:10566000F0904B04E114F10441F1C0904C04D0904F
:105670004D040E949D098C010C191D09C7010E944F
:10568000771480179107C8F480914A0490914B04D5
:105690009C013327887F9927892B09F077C04FE039
:1056A000429FC001439F900D11248E529C4FDC01FC
:1056B00014962C9122FF0E94BF1180911A0181152E
:1056C00019F1009135051091360501151105E1F02C
:1056D0000E949D09801B910B2091C8043091C90440
:1056E0002817390788F49091CB048091CA04981741
:1056F00009F44FC00E9401221092C9041092C804FC
:1057000010923605109235058091B30480FF1CC0BD
:105710008091190182FF18C00E949D09BC018091EF
:105720004E0490914F049B01281B390B809112016C
:10573000909113012817390738F041E08091500407
:10574000909151040E941E118091CE03811569F041
:105750000E949D092091CF033091D003821B930BAF
:105760008F3F9F4710F40E94B50CC4DA80910C0360
:10577000811551F08091060310920C03809307036A
:10578000809104038093050310E084C080E090E0E2
:105790008ECF0E94B02110923605109235050E94DE
:1057A000B308B2CF61E0812F0E944B08E82E60E081
:1057B000812F0E944B08EE0C8E29E12FF0E09F0113
:1057C00020503D4FD9014C91942F9370891709F4C3
:1057D00060C0A42FAA0FAA0F4A2F482BD9014C93BF
:1057E000CF0180579E4FDC012C91A42FAF70B0E009
:1057F000A058BE4FE350FD4F8C919081890F80835C
:10580000082E000C990B622F70E082179105DCF0D6
:105810002F2D30E0A9014F5F5F4F437055270417CC
:10582000150689F02C5F3C4F412F4F77D901149614
:105830004C9321E02F0D2370209306032091040345
:105840002F5F2093040322273327261B370B2817AB
:105850003907ECF0F09006032F2D30E0A9014F5FDF
:105860005F4F437055270417150689F02C5F3C4F96
:10587000412F4068D90114964C93A1E0AF0DA3705D
:10588000A0930603209104032F5F20930403D2D634
:1058900080831F5F00910703F0900603809103034C
:1058A000181708F47FCF90E00CEF7DEFF72E809172
:1058B000070320910603281709F443C0E82FF0E0FE
:1058C000E85FFC4F908197FBEE24E0F8192F1F77DB
:1058D0008F5F837080930703809105038F5F8093B0
:1058E000050397FD07C01BA70CA70E949D0953E065
:1058F000D52E06C01BA7FCA60E949D0962E0D62EED
:10590000BC018DA79EA7DFA6B1E0B8AB4BA55CA5F7
:105910008D2D91E00E94AE2219ABE11481F0FAAA1C
:105920000E949D09BC018BAB9CABDDAA1EAA49A9B4
:105930005AA98D2D90E00E94AE2291E0B8CF0AAB1B
:10594000EFCF91110E94A9090E940F0990910D03B8
:10595000891721F080930D030E94A90980912003EB
:10596000843009F0EDCD83E08093E9008091E80078
:1059700082FFE6CD8091E80090E085FF0BC00E9499
:105980002E0A40E2E42EF12C8E010F5F1F4F81158D
:1059900061F191E08091E8008B778093E8009115A8
:1059A00009F4CECD0091230310912403E981011560
:1059B000110549F1EE3F09F047C08A81833020F09C
:1059C0008550833008F040C0EA81EE3008F03CC0DA
:1059D000F0E0EB51FC4C41C68091F100F80181935D
:1059E0008F01F1E0EF1AF108A1F28091E80085FD46
:1059F000F3CF8091E8008B778093E8000E942E0A15
:105A0000811599F3C6CFE43148F4E11549F0E1502E
:105A1000E33130F4F0E0ED50FC4C1FC6EE3FA1F254
:105A20008FEF20C41A8289E08B830EC08A81823076
:105A300081F08330B1F0813099F70E94A90913D623
:105A40006B837C838D839E83CE0101960E947E0AA8
:105A500077CD88E290E044D61B821C821D828E8323
:105A6000F3CF80911E0390911F03892B69F38091DE
:105A70001A0390911B03A0911C03B0911D038B830B
:105A80009C83AD83BE83E0CF8A81823049F66B81EF
:105A90007C818D819E81E7D588E290E03DD6D4CF90
:105AA0004C816B818A810E945512982789279827FB
:105AB0009E838D83C9CF2D813E81322723273227B4
:105AC0004C816B818A810E94EF0BBECF0E947F13B5
:105AD000BBCF8A81823831F178F48038B1F08138D7
:105AE00009F0B2CF60E08B810E94F5068B818111B5
:105AF00016C00E94E906A8CF833809F0A5CF8B8194
:105B000020E0409115036C8106C08091130320E0D2
:105B10004B816091140390E00E94240795CF0E946E
:105B2000DB0692CFEB818FE7E43020F4F0E0ED5616
:105B3000FE4F80818093160380E00E94C90684CFC7
:105B40008A818238C1F050F4803891F0813809F0B0
:105B50007BCF809112038695869566CF833809F0B6
:105B600073CF809113038B83809114038C836CCF4C
:105B70008091150359CF80911603873230F08F350D
:105B800030F08E3930F482E04FCF80E04DCF81E0AD
:105B90004BCF83E049CF91D857CF80E18A8354CF50
:105BA00082E08A838FE540CF0C810D3108F04CCF25
:105BB0008A809B80982489249824A12CB12C9E0152
:105BC0002F5F3F4F7901020F132F111DE016F106D1
:105BD00009F43ACF80E03FE5831632E09306A10452
:105BE000B10420F4C4018F559E4F7AD5D701149685
:105BF0008C93BFEFEB1AFB0AEFEF8E1A9E0AAE0AE8
:105C0000BE0AE4CF80911E0390911F03892B09F4F3
:105C10001BCF8C818D3108F017CF882E912CA12CB1
:105C2000B12CCA80DB80DC24CD24DC24E12CF12CD7
:105C30008E010F5F1F4F412C512C32014814590423
:105C40006A047B0408F000CFFFE5CF16F2E0DF0620
:105C5000E104F10438F4D80114966C91C6018F5513
:105C60009E4F5AD5BFEF4B1A5B0A6B0A7B0AEFEFC8
:105C7000CE1ADE0AEE0AFE0A0F5F1F4FDFCF48D9A9
:105C8000E3CE84E08BCF8C818D3108F0DDCE882E81
:105C9000912CA12CB12CCA80DB80DC24CD24DC2407
:105CA000E12CF12C412C512C32018E010B5F1F4F46
:105CB000481459046A047B0408F0C6CE80E0F0E87A
:105CC000CF16D104E104F10418F4C601899608D571
:105CD000D8018D938D01BFEF4B1A5B0A6B0A7B0ACB
:105CE000EFEFCE1ADE0AEE0AFE0AE2CF2C81022F77
:105CF00010E02D3108F0A8CE8A819B819827892752
:105D000098272C01612C712C8038910508F09CCECD
:105D1000822E912CA12CB12C40E850E060E070E084
:105D2000441955096609770942175105610571053E
:105D300008F48ACE20911E0330911F03232B09F013
:105D40003EC01C01F9E22F0E311C80FBEE24FF2423
:105D5000E0F880FF0BC08896C3D49D8189279827DF
:105D6000892781159C4711F48FEF8D83D501C401DC
:105D7000840D951DA61DB71D80FF19C0680131E077
:105D8000C31AD108CE0105968C0D9D1D98AF8FAB1F
:105D9000C101800F911FA4D4AFA9B8AD9C9181150A
:105DA0009C4721F48FEFEFA9F8AD80838601FE01B7
:105DB0003196EE0DFF1D2FEFE016F10638F08E0143
:105DC0000F5F1F4FC12CD12C760124C09481858197
:105DD00081159C4711F42483258342E0E40EF11CD5
:105DE0003296EACF80E8481651046104710430F419
:105DF000D80114966C91C20189968ED4BFEFCB1A4C
:105E0000DB0AEB0AFB0AEFEF4E1A5E0A6E0A7E0A05
:105E10000F5F1F4FC814D904EA04FB0418F314CE13
:105E200080911E0390911F03892B09F40DCECE01A2
:105E300001960E947E0AFFEF21EE34E0F1502040EF
:105E40003040E1F700C0000047CB88E0EEE1F1E030
:105E5000DE01919601900D928A95E1F7FE0132964E
:105E60008FE1DF011D928A95E9F786E0898388E05A
:105E70007F96DE01159601900D928A95E1F7E4CDAB
:105E80008CE1898381E08A831B821C82DDCD8B813A
:105E90009C81092E000CAA0BBB0B35E0880F991FC3
:105EA000AA1FBB1F3A95D1F7AC01BD01405E5F4F01
:105EB0006F4F7F4F481759076A077B0708F4C4CD17
:105EC0008C31E1E09E07A105B10508F0BDCD4D3153
:105ED000F1E05F076105710520F04CE151E060E001
:105EE00070E0481B590BBC01645E7A4FCE010196ED
:105EF000C1D3AACD1B810C8140E0602F812F0E946D
:105F000083129827892798279A83898341E0602FF5
:105F1000812F0E9483129827892798279C838B833F
:105F200093CD8E819F819827892798270E94890782
:105F30009C0141E08D81811101C040E06C818B8129
:105F40000E94150C81CD4AE150E06FEF70E0CE0168
:105F50000796AFD380911E0389830A831B8282E058
:105F60008C831D8283E07BCD81E090E090932403BD
:105F70008093230382E390E09093110380931003B6
:105F80000E949D0990930F0380930E035DCD011530
:105F9000110571F1D0901A03E0900E03F0900F03F9
:105FA0000E949D098E199F098536910540F1D3FE07
:105FB00026C0D2FE24C00E949D0990930F038093B7
:105FC0000E03809110039091110301979093110398
:105FD00080931003892B61F4109224031092230301
:105FE00081E090E090931F0380931E0300E010E097
:105FF00080911E0389830A838091100315CD82E36B
:1060000090E09093110380931003F2CF10921F033E
:1060100010921E0319CD0B811C8140E250E06FEFFE
:1060200070E0CE01019645D320E534E042E050E037
:1060300080E090E0F901659175910617170740F42B
:10604000DE0111968A0F9B1FFC0171836083CA01D8
:10605000F5E020313F0709F4F7CCAC014E5F5F4F0C
:10606000245F3F4F4132510528F3EECC4B815C81D8
:1060700080E594E02CE135E0FC01659175914617CF
:10608000570709F4E0C00C9628173907A9F7C8CCC0
:106090008B819C8100E514E0F8012591359128174A
:1060A000390709F4E1C0045F1F4FF5E00C311F0709
:1060B00099F7EE24EA94FE2CF2C00E942212C4CC7E
:1060C0008B81823009F450C078F4811136C0FE0112
:1060D00033968DE1DF011D928A95E9F788E0898387
:1060E0008A8383E088A3B0CC833009F472C0843003
:1060F00009F0AACC1C818AE0FE013596DE0191965A
:1061000001900D928A95E1F789A59AA50E948907C9
:106110009AA789A78FEF183060F4FAE01F9FB001AB
:1061200011246F5A7E4F4AE050E0CE01819612D37F
:1061300080E089830E941E1487CC8C819AE0F92E1E
:106140008E010F5D1F4FF8012F2D11922A95E9F74F
:10615000B8010E9462148983F801DE011296019051
:106160000D92FA94E1F770CC1C818AE0FE0135961D
:10617000DE01919601900D928A95E1F789A19AA18D
:106180000E9489079AA389A38BA19CA10E948907D9
:106190009CA38BA38DA19EA10E9489079EA38DA382
:1061A0008FA198A50E94890798A78FA38FEF183019
:1061B00060F43AE0139FB00111246F5F7E4F4AE014
:1061C00050E0CE018196C6D280E089830E94960776
:1061D0003BCC2C816AE0CE018196DC01E62F1D923A
:1061E000EA95E9F7283080F4629FB00111246F5AD4
:1061F0007E4F4AE050E064D280E089838AE0FE016D
:10620000B196DE01129637CE8FEFF7CF8091F7026D
:10621000811509F416CAB0E1B9BDE2E1E9BD09B4DE
:1062200000FEFDCF8091D8008F7D8093D8008091B3
:10623000E00082608093E0008091E00081FDFCCF6F
:106240000E94CE0DFEC9FC0136962591359121158F
:10625000310509F4E5CB4FE150E0BE016E5F7F4FA1
:10626000F90109958983F0CBF8013896259135918C
:106270002115310509F41DCF4CE150E0BE016B5FE3
:106280007F4FC801F90109957C01892B41F4F80180
:106290003A9685919591009711F0FC010995E98254
:1062A000D3CB1F921FB61F9211248F939F93AF934E
:1062B000BF938091F602811113C0809144029091A6
:1062C0004502A0914602B09147024196A11DB11D21
:1062D0008093440290934502A0934602B0934702F4
:1062E000BF91AF919F918F911F901FBE1F901895E6
:1062F00078941F921FB61F9211248F939F93AF9390
:10630000BF938091440290914502A0914602B091C2
:1063100047020196A11DB11D80934402909345024E
:10632000A0934602B0934702BF91AF919F918F9186
:106330001F901FBE1F9018951F920F920FB60F92BD
:1063400011242F933F934F935F936F937F938F937A
:106350009F93AF93BF93EF93FF938091E10082FFF0
:1063600009C08091E20082FF05C08091E1008B7F2F
:106370008093E1008091DA0080FF24C08091D800F2
:1063800080FF20C08091DA008E7F8093DA008091B8
:10639000D90080FFA9C080E189BD82E189BD09B42F
:1063A00000FEFDCF81E080932003809133028111B4
:1063B00009C00E945F0A0E94BC0A8091E2008460CA
:1063C0008093E2008091E10080FF1AC08091E2009A
:1063D00080FF16C08091E2008E7F8093E200809162
:1063E000E20080618093E2008091D8008062809317
:1063F000D80019BC85E08093200383E080931701C7
:106400008091E10084FF2FC08091E20084FF2BC0C7
:1064100080E189BD82E189BD09B400FEFDCF809194
:10642000D8008F7D8093D8008091E1008F7E80938B
:10643000E1008091E2008F7E8093E2008091E20093
:1064400081608093E20080913202811509F452C08C
:1064500084E08093200380912003843009F052C0AF
:1064600082E0809317018091E10083FF2CC080912E
:10647000E20083FF28C08091E100877F8093E100E4
:1064800082E080932003109232028091E1008E7F9F
:106490008093E1008091E2008E7F8093E200809102
:1064A000E20080618093E20042E060E080E00E94D0
:1064B0008C0A8091F00088608093F00081E08093E6
:1064C000170180931601FF91EF91BF91AF919F91BA
:1064D0008F917F916F915F914F913F912F910F908D
:1064E0000FBE0F901F90189519BC109220031092A8
:1064F000330268CF8091E30087FF02C083E0A9CF19
:1065000081E0A7CF81E0ADCF1F920F920FB60F921F
:106510001124EF92FF920F931F932F933F934F936A
:106520005F936F937F938F939F93AF93BF93CF931B
:10653000EF93FF9309EE10E0F8018081C091EC0029
:106540008F70C795CC27C795C82B108280EFE82E97
:10655000F12CF7018081877F808378940E943A0E26
:10656000F8011082F701808188608083CF70F80184
:10657000C083FF91EF91CF91BF91AF919F918F9188
:106580007F916F915F914F913F912F911F910F914B
:10659000FF90EF900F900FBE0F901F9018952F92C5
:1065A0003F924F925F926F927F928F929F92AF92A3
:1065B000BF92CF92DF92EF92FF920F931F93CF93F0
:1065C000DF93CDB7DEB7CA1BDB0B0FB6F894DEBF87
:1065D0000FBECDBF09942A88398848885F846E84AD
:1065E0007D848C849B84AA84B984C884DF80EE80F7
:1065F000FD800C811B81AA81B981CE0FD11D0FB600
:10660000F894DEBF0FBECDBFED010895AA1BBB1BE2
:1066100051E107C0AA1FBB1FA617B70710F0A61BA2
:10662000B70B881F991F5A95A9F780959095BC01C3
:10663000CD01089597FB072E16F4009406D077FD40
:1066400008D0E4DF07FC05D03EF4909581959F4F7C
:106650000895709561957F4F0895EE0FFF1F059087
:10666000F491E02D099469279627692778278727D1
:1066700078270895FB01DC0102C005900D9241507E
:106680005040D8F70895FB01DC0104C08D910190C2
:10669000801921F441505040C8F7881B990B089588
:1066A000FB01DC0102C001900D9241505040D8F72F
:1066B0000895DC0101C06D9341505040E0F708950A
:1066C000DC01CB01FC01F999FECF06C0F2BDE1BDB2
:1066D000F89A319600B40D9241505040B8F70895A1
:1066E000F999FECF92BD81BDF89A992780B508959A
:1066F000A8E1B0E042E050E0E5CFDC01A40FB51F17
:106700004150504040F0CB01840F951F2E9105D091
:1067100041505040D8F70895262FF999FECF92BDE9
:1067200081BDF89A019700B4021639F01FBA20BD56
:106730000FB6F894FA9AF99A0FBE08950396272F88
:10674000ECDFEADF252FE9DF242FE7CF0196272FA3
:10675000E4DFE2CFDC01CB0102C02D9105D0415036
:106760005040D8F70895262FF999FECF1FBA92BD51
:1067700081BD20BD0FB6F894FA9AF99A0FBE019622
:106780000895F894FFCF170F3D0F430F3D0F430FB0
:10679000950FB60F430FBC10C910A419A719D21931
:1067A000AC19D719B119DC19B619E119BB19E619D9
:1067B000C919CF19A419A719D219AC19D719B11928
:1067C000DC19B619E119BB19E619252F402F472FFF
:1067D0007A2F912FA32FB42FC72F06300B303630CE
:1067E00048305D306030122D162D442D502D5B2D1C
:1067F000662D692DA02DCB2D102D102FCD2DD02D38
:0C680000D42D022E3F2E412E432E762E6A
:10680C0000FF00FFFF039A09CF0BE50BB509EA0B5C
:10681C00C60BAF000000010001010100FFFFC02A00
:10682C00CAFEC35E1F410044226D3B011901AC003E
:10683C0041025A027A02F5C633F6F0320302010025
:10684C00040506070B0A0908FFFFFFFF03000200FF
:10685C000100000000010101020103010302020218
:10686C0001020002040404040404040404040404E7
:10687C00003131295A1B750A94973435676696F4A2
:10688C0000FF0100010000FFFF0000010001FF00FC
:10689C000404020F3F7FBDE200E900EA00B500B638
:1068AC0000B700CD008301CC008A01920194012134
:1068BC0002230224022502260227022A02B300B474
:1068CC00006F0070009F01CB019F02A002E200E963
:1068DC0000EA00B500B600B700CD008301CC008AF9
:1068EC00019201940121022302240225022602278F
:1068FC00022A02B300B4006F0070009F01CB019F0D
:04690C0002A00200E3
:00000001FF
